:1000000053C1000079C1000077C1000075C1000034
:1000100073C1000071C100006FC100006DC100001C
:100020006BC1000069C1000067C1000065C100002C
:1000300063C1000061C100005FC100005DC100003C
:100040000C94372C59C100000C944C1F55C1000072
:1000500053C1000051C100004FC100004DC100005C
:100060000C94A81249C1000000008207330FC71684
:10007000331EAD254F2D0A35D93CB6449C4C8554D2
:100080006C5C4A64196CD4737B7B0B83848AE49127
:100090002C995AA06FA765AE3CB5F0BB7EC2E7C8ED
:1000A0000000B200F9010F03E703A5043C05C405F5
:1000B0003806A306F9064907D10FAC0F680FFB0EEF
:1000C000580E770D550CFB0A810905089E0666053A
:1000D00061048303D4024602DA0183013F01070170
:1000E000DA00B6002000327DFF1F1F1F0000000055
:1000F0000000000000001F1F1F1F1F1F0000001F27
:100100001F0000000E0E0E0C080000000000001F73
:100110001F00000000030F0F1F000000001F1F1F23
:100120001F00000000181E1E1F1F0F0F03000000FD
:10013000001F1E1E18000000001F1F1F1F000000D0
:10014000000E0E0E0E0C0800000000000000001F44
:100150001F1C1C1C1E1E1F1F1F0707070F0F1F1F22
:100160001F1F1F1F1C1C1C1C1C181C1E0F07070711
:10017000071F1D1D1C1C1C1C1C1F1717070707072A
:10018000071C1C1C1C1C1F1F1F070707070F1E1C1A
:10019000181F0000000000001F1F00000E000000DC
:1001A0001F1F00040E0400001F1F0E1F1F1F1F0E25
:1001B0001F101010101010101018181818181818F8
:1001C000181C1C1C1C1C1C1C1C1E1E1E1E1E1E1E65
:1001D0001E000000000000001F0000000000001FC3
:1001E0001F00000000001F1F1F000000001F1F1F36
:1001F0001F0000001F1F1F1F1F00001F1F1F1F1FAA
:100200001F001F1F1F1F1F1F1F4253543A00525031
:100210004D3A004C414D4244413A0043543A005457
:1002200048523A004C4D4D3A202020202020414792
:10023000543A004C443A2020202020202052504D97
:100240003A004D6178200000000000240027002AB9
:100250000000000000250028002B00000000002303
:100260000026002900040404040404040402020219
:1002700002020203030303030301020408102040E7
:100280008001020408102001020408102000000070
:100290000700020100000304060000000000000047
:1002A0000000010E3111CE2011241FBECFEFD8E087
:1002B000DEBFCDBF13E0A0E0B1E0ECE3F5E702C0A4
:1002C00005900D92AC3BB107D9F715E0ACEBB3E06C
:1002D00001C01D92AD3AB107E1F712E0C8EAD2E0E1
:1002E00004C02297FE010E943F36C23AD107C9F7E7
:1002F0000E940E0E0C949C3A83CE08950895FC0142
:1003000020E030E040E050E080E6848B81EE858B99
:1003100080E090E0A0E8BFE382839383A483B58369
:1003200081E0838B26833783408751871286118231
:10033000108280E090E0A0ECB2E483879487A587E8
:10034000B6872787308B418B528B0895CF93DF93ED
:10035000EC018B89861709F43FC06B8B6130A1F4E7
:1003600080E090E0A0E8BFE38A839B83AC83BD83F9
:100370006F85788989899A8920E030E040E050E0F3
:100380000E94E0316C8913C080E090E0A0ECBFE3F4
:100390008A839B83AC83BD836F85788989899A8999
:1003A00020E030E040E050E00E94E0316D89181616
:1003B00054F470E080E090E00E940C336F87788BFB
:1003C000898B9A8B09C070E080E090E00E940C332A
:1003D0006B877C878D879E87DF91CF910895EF9201
:1003E000FF920F931F93CF93DF93EC0180910E0444
:1003F00090910F040097E9F46F85788989899A892B
:1004000020E030E040E050E00E94B531882371F5F3
:100410008B859C85AD85BE858F87988BA98BBA8B84
:1004200080E090E0A0E0B0E08B879C87AD87BE873E
:100430001DC018161906D4F4EF84F88809891A89A2
:10044000C801B70120E030E040E050E00E94E03118
:10045000181664F4EB86FC860D871E8780E090E01A
:10046000A0E0B0E08F87988BA98BBA8BDF91CF91FA
:100470001F910F91FF90EF900895FC0180818130D2
:1004800031F0813010F01082089581E001C082E0E7
:1004900080830895EF92FF920F931F93CF93DF9382
:1004A000C0E0D0E0FE01EE0FFF1FE859FF4F0591BD
:1004B00014916017710708F437C021969E01220F2E
:1004C000331F2197F901E859FF4F859194918617C1
:1004D000970750F1F901E859FF4FE590F490601B40
:1004E000710B80E090E022E330E040E050E00E94B9
:1004F0007735E01AF10A00E010E0A80197010E94A8
:10050000D73582E390E0C89FA001C99F500DD89FC6
:10051000500D1124420F531FCA01DF91CF911F913B
:100520000F91FF90EF9008952196CC31D10509F0FD
:10053000B9CF40E050E0F0CFCF92DF92EF92FF9240
:100540000F931F93CF93DF9320E030E0F901EE0F7C
:10055000FF1FE854FF4FC591D491C617D70708F481
:1005600045C069010894C11CD11C7601EE0CFF1C2A
:10057000F701E854FF4F8591949168177907B0F11E
:10058000F701E854FF4F05911491601B710B80E057
:1005900090E026EF3FEF4FEF5FEF0E947735C01BF3
:1005A000D10B9E0140E050E00E94D735C60143E0E8
:1005B000880F991F4A95E1F78E0D9F1D820F931F9B
:1005C0004E9723E0883E920714F087EE93E02FEFDA
:1005D000883D920714F488ED9FEFDF91CF911F9132
:1005E0000F91FF90EF90DF90CF9008952F5F3F4FD6
:1005F0002631310509F0AACF80E090E0E1CFCF921B
:10060000DF92EF92FF920F931F93CF93DF93C0E09F
:10061000D0E06E01CC0CDD1CF601E056FF4F0591D9
:1006200014916017710708F442C021969E01220FB1
:10063000331F2197F901E056FF4F8591949186175A
:100640009707A8F1F901E056FF4FE590F490601B81
:10065000710B80E090E02AE030E040E050E00E9442
:100660007735E01AF10A00E010E0A80197010E9436
:10067000D735CE01B3E0880F991FBA95E1F78C0DFD
:100680009D1D820F931F0A9723E0883E920714F066
:1006900087EE93E097FF02C080E090E0DF91CF917A
:1006A0001F910F91FF90EF90DF90CF9008952196CA
:1006B000CC30D10509F0ADCF80E090E0E4CF70E020
:1006C000FB01F6962CEB33E0EE0FFF1FE20FF31F5A
:1006D0008091EA039091EB0391838083FB017D96E7
:1006E000EE0FFF1FEE0FFF1FE20FF31F8091FE03BF
:1006F0009091FF03A0910004B09101048083918345
:10070000A283B383FB01B196EE0FFF1FEE0FFF1F15
:10071000E20FF31F80910C0490910D04AA2797FD1E
:10072000A095BA2F80839183A283B3836B5D7F4FA3
:10073000FB01EE0FFF1FEE0FFF1FE20FF31F809173
:10074000140490911504A0911604B09117048083AD
:100750009183A283B383635D7F4F660F771F260F5C
:10076000371F80911E0490911F04F90191838083AB
:10077000089580916C04823001F1833020F481303F
:1007800009F041C005C0873021F18830E1F532C061
:1007900080E090E0A0E0B0E08093E2039093E30378
:1007A000A093E403B093E5038091E8039091E903FB
:1007B0009093E7038093E603089588E694E00E940F
:1007C000D91984EE94E069E670E040916D040C94D0
:1007D000E60E88E694E066E00E945D14FC01009756
:1007E00091F01286118688E893E194878387CF0180
:1007F0000C94751D88E694E067E00E945D140097F4
:1008000011F00C94721E089520916C04223029F08E
:10081000233049F0213041F430CE80916C04909126
:100820006D040C94F01B29CE08950F931F938C0137
:1008300088E694E00E94761B0E947F2C605F784DD2
:100840008F4F9F4FF80164837583868397831F9131
:100850000F91089520910C0430910D04C901805727
:100860009741855F914020F483E068E270E007C023
:1008700089E1243638072CF083E06FEF70E00C94A8
:10088000412D205737412CF483E060E070E00C9458
:10089000412D0895DF92EF92FF920F931F93CF9314
:1008A000DF93EC01D0906D042091EA033091EB03CB
:1008B0008091EC039091ED03815B94401CF4215BEB
:1008C000344054F00E947F2C68577C4E8F4F9F4FCE
:1008D0006E877F87888B998BEE84FF8408891989BE
:1008E0000E947F2CE616F70608071907E0F0EA8851
:1008F000FB880C891D890E947F2C6E157F0580075F
:100900009107E8F0DD2019F492E0D92E01C0DD2432
:100910000E947F2C6C597F4F8F4F9F4F6A8B7B8B30
:100920008C8B9D8B07C084EE94E069E670E00E949A
:10093000EA0ED82E88E694E06D2D0E94CB1988E649
:1009400094E06D2D0E94CB19DF91CF911F910F91F3
:10095000FF90EF90DF900895AF92BF92CF92DF9219
:10096000EF92FF920F931F938091020490910304E2
:10097000A0910404B09105048093DE039093DF03FB
:10098000A093E003B093E10300D000D06091BE03D8
:100990007091BF03882777FD8095982F28EC30E071
:1009A00040E050E0EDB7FEB72183328343835483A8
:1009B00020E030E040E050E0E12CE0E1FE2E012DAF
:1009C000112DAA24BB2465010E94D3232AE030E024
:1009D00040E050E00E94D7353093E9032093E803CC
:1009E0000F900F900F900F9084EE94E06DEC70E0FC
:1009F000422F0E94E60E6091DE037091DF0380912A
:100A0000E0039091E10320E030E04AE754E40E94E3
:100A100019300E94BB32AB01BC0188EC90E00E940F
:100A2000A90E80E090E0A0E0B0E08093E203909314
:100A3000E303A093E403B093E5038091E80390916E
:100A4000E9039093E7038093E6030CE815E0C801FF
:100A500060E071E00E94D822C80162E071E00E946B
:100A60003F214091DE035091DF036091E0037091DC
:100A7000E103C80122E030E00E94CA231F910F91D8
:100A8000FF90EF90DF90CF90BF90AF9008959C01C2
:100A900080916C04813011F4C9015ECF0895CF9329
:100AA000DF93EC01605870406230710529F16330CA
:100AB000710509F444C06130710509F044C08AA988
:100AC0009BA9ACA9BDA90097A105B10519F4CE0158
:100AD0009BDE2EC00E947F2C2AA93BA94CA95DA9B0
:100AE00028513C4F4F4F5F4F62177307840795079C
:100AF00050F1CE019ADE1CC08AA99BA9ACA9BDA960
:100B00000097A105B10519F4CE0133DE11C00E9492
:100B10007F2C2AA93BA94CA95DA928513C4F4F4FD6
:100B20005F4F621773078407950768F0CE01AFDF48
:100B30000E947F2C6AAB7BAB8CAB9DAB04C01AAA26
:100B40001BAA1CAA1DAADF91CF9108950F931F9392
:100B5000DF93CF9300D0CDB7DEB78C01FC0180814D
:100B6000833009F45EC08CE895E06DE071E00E948E
:100B70003F218CE895E06FE071E00E943F214091B9
:100B8000D0045091D1046091D2047091D3048CE8C8
:100B900095E022E030E00E94C9238CE895E060E017
:100BA00071E00E943F214091FE035091FF0360914C
:100BB0000004709101048CE895E022E030E00E948E
:100BC000C9238CE895E060E071E00E943F214091EC
:100BD000D9045091DA046091DB047091DC048CE854
:100BE00095E022E030E00E94C9238CE895E060E0C7
:100BF00071E00E943F218091CE049091CF04892B17
:100C000031F48CE895E064E171E00E943F218CE8CA
:100C100095E06DE171E00E943F218CE895E00E9433
:100C20008B228CE895E06DE071E00E943F21F80195
:100C30008081813049F0813008F499C1823079F1A6
:100C4000833009F092C149C1F80140855185628520
:100C500073858CE895E02AE030E00E9406228CE85B
:100C600095E06FE171E00E943F210EEB13E0F80187
:100C7000619171918F018CE895E04AE050E00E940B
:100C800068228CE895E06FE171E00E943F21F3E07B
:100C90000C3D1F0761F7F8016081718117C18CE875
:100CA00095E062E070E04AE050E00E9468228CE843
:100CB00095E061E271E00E943F21F8014085518595
:100CC000628573858CE895E02AE030E00E94062278
:100CD0008CE895E06FE171E00E943F2160910C0487
:100CE00070910D048CE895E04AE050E00E94682283
:100CF0008CE895E06FE171E00E943F214091FE0396
:100D00005091FF0360910004709101048CE895E01C
:100D100022E030E00E94C9238CE895E06FE171E0A9
:100D20000E943F2160910E0470910F048CE895E0C1
:100D30004AE050E00E9468228CE895E06FE171E0A3
:100D40000E943F21409106045091070460910804DD
:100D5000709109048CE895E022E030E00E94C923FC
:100D60008CE895E06FE171E00E943F21409114040E
:100D70005091150460911604709117048CE895E069
:100D800022E030E00E94C9238CE895E06FE171E039
:100D90000E943F214091100450911104609112046F
:100DA000709113048CE895E022E030E00E94C923A2
:100DB0008CE895E06FE171E00E943F216091EA03C9
:100DC0007091EB038CE895E04AE050E00E946822C5
:100DD0008CE895E06FE171E00E943F216091EC03A7
:100DE0007091ED038CE895E04AE050E00E946822A3
:100DF0008CE895E06FE171E00E943F21409124046E
:100E00005091250460912604709127048CE895E0A8
:100E100022E030E00E94C9238CE895E06FE171E0A8
:100E20000E943F2160911E0470911F048CE895E0A0
:100E30004AE050E00E9468228CE895E06FE171E0A2
:100E40000E943F2160912004709121048CE895E07C
:100E50004AE050E00E9468228CE895E06FE171E082
:100E60000E943F2160912204709123048CE895E058
:100E70004AE050E00E9468228CE895E06FE171E062
:100E80000E943F2160911804709119048CE895E04C
:100E90004AE050E00E9468228CE895E06FE171E042
:100EA0000E943F2160911A0470911B048CE895E028
:100EB0004AE050E00E9468228CE895E06FE171E022
:100EC0000E943F2160911C0470911D048CE895E004
:100ED0004AE050E00E9468224AC08CE895E06CE04D
:100EE00074E042E050E00E9420218CE895E06EE042
:100EF00074E042E050E00E9420216091060470916D
:100F000007048091080490910904C1D69A838983CB
:100F10008E010F5F1F4F8CE895E0B80142E050E072
:100F20000E942021609102047091030480910404C6
:100F300090910504ACD69A8389838CE895E0B8013A
:100F400042E050E00E9420218CE895E06AEE73E0D8
:100F500042E050E00E9420218CE895E06CEE73E0C6
:100F600042E050E00E94202102C0F80110828CE88B
:100F700095E06DE171E00E943F218CE895E00E94D0
:100F80008B2260D6BC018CE895E04AE050E00E94DC
:100F9000A9220F900F90CF91DF911F910F9108958B
:100FA000EF92FF920F931F9384EE94E069E670E056
:100FB00011D7682F88E694E00E94CB1984EE94E064
:100FC0006DEC70E007D7853128F490E09093E90349
:100FD0008093E80388EC90E073D60E94613220E0B1
:100FE00030E04AE754E40E940E317B018C0120E09E
:100FF00030E040E050E00E94E031181694F4C8015F
:10100000B7012AE939E949E95FE30E9436328823CA
:1010100044F4E092DE03F092DF030093E0031093C8
:10102000E1031F910F91FF90EF900895DF92EF92EF
:10103000FF920F931F93CF93DF938C017C01C0E04D
:10104000D0E0DD24DA9410C08CE895E00E948B207B
:10105000D82E06C08CE895E00E948B20F701818F86
:1010600021960894E11CF11C8CE895E00E94602018
:10107000892B31F0C931D10531F0209729F3EACF1E
:10108000C931D10589F5F1E0FD1570F1F801628DE6
:10109000738D848D958D0E94613220E030E04AE7A7
:1010A00054E40E940E316093D0047093D104809375
:1010B000D2049093D304DD2009F05AC0F80162A154
:1010C00073A184A195A10E94613220E030E04AE73B
:1010D00054E40E940E316093D9047093DA04809333
:1010E000DB049093DC0444C0F3E0DF1619F184E0E4
:1010F000D81671F1E2E0DE1609F03AC02297C4F189
:10110000F801828D823069F0833018F4813081F5E6
:1011100005C0833049F0843059F509C0C80174DB3B
:1011200027C0C80182DB24C0C80123DB21C0C8015D
:10113000AEDC1EC02297E4F0F801828D823029F0E7
:101140008330B1F4F801D08213C0F801808310C05D
:10115000C230D1056CF0F801828D843049F42497B7
:101160003CF0F801838D8093E204848D8093E30446
:101170008CE895E00E94AF20DF91CF911F910F91F5
:10118000FF90EF90DF900895CF93DF93EC012D96C1
:10119000CE0160E270E041E050E00E94A211CE0179
:1011A0000E94D810882319F0CE010E94DE10DF9132
:1011B000CF910895CF93DF93EC012D96CE0161E29C
:1011C00070E041E050E00E94A211CE01F1D78823E7
:1011D00011F0CE01F3D7DF91CF910895FF920F93D5
:1011E0001F93F62E8C01035F1F4FC80160E270E071
:1011F000DED7C8016F2D0E943211C8010E948311F1
:101200001F910F91FF900895FF920F931F93F62E59
:101210008C01035F1F4FC80161E270E0C8D7C801AD
:101220006F2D0E943211C8010E9483111F910F91EE
:10123000FF900895CF92DF92EF92FF920F931F934A
:10124000CF93DF938C01D62EFC018485F8E0F6174E
:1012500030F48D77F8018487862F885004C08E770C
:10126000F8018487862F90E00197B3E0880F991FDB
:10127000BA95E1F7A0ECCA2EC82AC801F801648526
:10128000ADDFC7E0D0E0F1E0EF2EF12CC7010C2E6E
:1012900002C0880F991F0A94E2F76C2D682381E140
:1012A0000E94F22D8DE061E00E94F22D8DE060E061
:1012B0000E94F22D2197C230D10541F78DE061E007
:1012C0000E94F22D8DE060E00E94F22D8DE061E041
:1012D0000E94F22D8DE060E00E94F22DEE24FF24AA
:1012E000CBE0D0E08CE00E94262E0C2E02C0880FAE
:1012F000991F0A94E2F7E80EF91E8DE061E00E9462
:10130000F22D8DE060E00E94F22D2197FFEFCF3F9C
:10131000DF0741F7F8018485F8E0FD1510F48268D5
:1013200001C08168F8018487C801F801648556DF2F
:10133000C701DF91CF911F910F91FF90EF90DF9048
:10134000CF900895AF92BF92CF92DF92EF92FF922B
:101350000F931F93DF93CF93CDB7DEB760970FB690
:10136000F894DEBF0FBECDBF7C01DE011196E5E330
:10137000F1E080E101900D928150E1F7CC24DD2471
:101380005E010894A11CB11CF501EC0DFD1D8081CE
:101390009181880F991F880F991FF7016485637EDB
:1013A000682B6487C7011ADF64E170E080E090E099
:1013B0000E94B32CC70160E13DDFAA2797FDA095ED
:1013C000BA2FBC01CD010E94613220E030E040EA3A
:1013D00050E40E94193020E030E040E859E30E94D8
:1013E000193020E030E44CE156E40E9419300E94AC
:1013F000552E9B01AC01C701B9014CD88C01F4E01A
:1014000082399F0718F060E070E00CC06091100412
:101410007091110480911204909113040E94BB32C8
:10142000600F711FF601E454FC4F77A766A7809107
:101430002E0490912F046817790718F0C70163E014
:101440003ED982E090E0C80ED91E94E0C916D104BE
:1014500009F09ACF60960FB6F894DEBF0FBECDBFED
:10146000CF91DF911F910F91FF90EF90DF90CF9080
:10147000BF90AF900895AF92BF92CF92DF92EF925C
:10148000FF920F931F93CF93DF93EC016091BE0304
:101490007091BF03882777FD8095982F0E94613255
:1014A00020E030E040EA50E40E94193020E030E0D3
:1014B00040E859E30E94193020E030E048E452E46B
:1014C0000E94193020E030E040E251E40E94C72F32
:1014D00020E030E048EC52E40E940E3160930204B8
:1014E0007093030480930404909305042091DE0319
:1014F0003091DF034091E0035091E1030E94C72F38
:101500006093FE037093FF038093000490930104A3
:1015100020913404309135044091360450913704C1
:101520000E940B3288231CF0CE0161E0C8D8E09005
:10153000D203F090D3030027F7FC0095102FC801C9
:10154000B7010E94613220E030E040E859E30E9498
:10155000193020E030E040EA50E40E9419309B014D
:10156000AC010E94F22F20E030E040E251E40E9402
:10157000F22F23E333E34BE651E40E940E316093F4
:10158000060470930704809308049093090400D024
:1015900000D088EC90E0A0E0B0E0EDB7FEB781832A
:1015A0009283A383B483C801B70120E030E040E018
:1015B00050E0E12CF0E1FF2E012D112DAA24BB24D7
:1015C00065010E94D3230F900F900F900F90693CFC
:1015D000710514F068EC70E077FF02C060E070E025
:1015E00070930B0460930A046091100470911104CD
:1015F000809112049091130426E636E646E65FE3F6
:101600000E9419307B018C016091DA037091DB0339
:10161000882777FD8095982F0E94613220E030E086
:101620004AEF53E40E94193020E030E040E859E3EB
:101630000E9419302DEC3CEC4CEC5DE30E9419301B
:101640009B01AC01C801B7010E94F22F6093100406
:1016500070931104809312049093130400D000D06F
:101660006091D4037091D503882777FD8095982FDA
:1016700024E630E040E050E0EDB7FEB7218332834E
:10168000438354832CE632E040E050E0EAECEE2E57
:10169000EDE0FE2E012D112DAA24BB2465010E9430
:1016A000D3230F900F900F900F906536710514F0B3
:1016B00064E670E077FF02C060E070E084E690E0EE
:1016C000861B970B90930F0480930E046091D803B0
:1016D0007091D903882777FD8095982F0E946132F9
:1016E00020E030E040EA50E40E94193020E030E091
:1016F00040E859E30E941930609314047093150474
:1017000080931604909317046091FA037091FB0381
:101710002091F8033091F903F901EE0FFF1FE25118
:10172000FC4F408151818091D6039091D7039183E2
:101730008083680F791F641B750B7093FB036093A4
:10174000FA032F5F3F4F3093F9032093F8032530BE
:10175000310524F01092F9031092F803CB0165E0F3
:1017600070E00E94A2357093FD036093FC0388270C
:1017700077FD8095982F0E9461322FE832EC45E189
:1017800050E40E9419300E94BB3270930D046093A4
:101790000C04882777FD8095982F2091480430917C
:1017A000490440914A0450914B046217730784071F
:1017B000950724F0CE0162E00E945F0380E00E9462
:1017C0001F2DAA2797FDA095BA2FBC01CD010E941D
:1017D000613220E030E040EA50E40E94193020E01D
:1017E00030EC4FE754E40E940E3128E431EE42E839
:1017F00050E40E94193023E333E343E35FE30E94A4
:10180000F22F609324047093250480932604909310
:1018100027048A81813011F4CE0194DD6091C203E6
:101820007091C303CE010E949C029093190480938F
:1018300018046091C4037091C503CE010E949C02FC
:1018400090931B0480931A046091C6037091C703A0
:10185000CE010E949C0290931D0480931C04609111
:10186000C8037091C903CE010E94FF0290931F0428
:1018700080931E046091CA037091CB03CE010E9435
:10188000FF0290932104809320046091CC03709117
:10189000CD03CE010E94FF02909323048093220483
:1018A000DF91CF911F910F91FF90EF90DF90CF903C
:1018B000BF90AF900895EF92FF921F93CF93DF9365
:1018C000EC010E947F2C688779878A879B87AEEB23
:1018D000EA2EA3E0FA2E11E0CE01612FABDCF70176
:1018E000819391937F011F5F1131B1F7CE01C3DD69
:1018F000CE010E942A0488E694E00E945C1BCE017F
:1019000059DC682F70E0CE01CAD80E947F2C2C8150
:101910003D814E815F81621773078407950778F0D8
:1019200084EE94E064E670E040916C044FD280EC69
:101930009FE1A8E9B9E18C839D83AE83BF838FE0EB
:101940000E94262EBC018EEC94E00E94A6018EEC33
:1019500094E00E94EF016091D9047091DA048091C3
:10196000DB049091DC040E94BB329B01AC018BE054
:10197000B9010E94412D0E947F2C2E893F89488DFC
:10198000598D261737074807590778F4CE014EDBE3
:10199000CE01DCD88E899F89A88DB98D4496A11D72
:1019A000B11D8E8B9F8BA88FB98FDF91CF911F9127
:1019B000FF90EF9008950D96EFC30D96EDC3EF9253
:1019C000FF920F931F93DF93CF930F92CDB7DEB7A4
:1019D0007C018FEFF7018487CE010196DDD3F701FB
:1019E00016861786108A118A128A138A148A158A13
:1019F000148215821682178210861186128613862B
:101A000080E090E0A0E0B0E08093E2039093E303F5
:101A1000A093E403B093E5031092E7031092E6036A
:101A200081E08383808312AA13AA14AA15AA85E0F1
:101A300061E00E949F2D8FE060E00E949F2D8FE06B
:101A400061E00E94F22D8BE061E00E949F2DE1EBAE
:101A5000F0E080818760808381E161E00E949F2DBA
:101A60008CE060E00E949F2D8DE061E00E949F2D40
:101A700081E160E00E94F22D8DE060E00E94F22D95
:101A80000CE815E0C80140E051EE60E070E00E9413
:101A9000DD1FC7010D9657D4C701F70164859EDB92
:101AA000C80163E271E00E94D822C70179DA08E632
:101AB00014E0C80160ED77E00E94E419C8010E94BB
:101AC000691BC70163E8A0DB0E947F2CF701668BCE
:101AD000778B808F918F0F90CF91DF911F910F9116
:101AE000FF90EF90089508950895CF93DF93EC0150
:101AF00080E090E0FE01E80FF91F1182108202964B
:101B000082329105B9F780E090E0A0E8BFE38AA3B4
:101B10009BA3ACA3BDA380E090E0A0E0B0E08EA3C7
:101B20009FA3A8A7B9A71BA61AA61DA61CA61DAEF3
:101B30001CAE1FAE1EAEC05CDF4F19921992899386
:101B40009993A993B99388839983AA83BB83289691
:101B500019821882BA93AA939A938A932696199215
:101B600019921992199289939993A993B993899388
:101B70009993A993B993199219921992199219925A
:101B8000199219921992199219921992199288839D
:101B90009983AA83BB83C856D040DE01A459BF4FA6
:101BA000FE01EC58FF4F80E090E020E030E040E0A4
:101BB00050E011961C921E922083318342835383FE
:101BC000108A118A128A138A20A331A342A353A335
:101BD000D9961C921E92D89701961296349684300C
:101BE000910539F71BAA1AAA1DAA1CAA1FAA1EAA88
:101BF00019AE18AE1BAE1AAE1FA61EA6DF91CF916E
:101C000008958CEB93E070DF88E694E055D688E980
:101C100094E0D1DE8EEC94E00C947E010E94E12CE5
:101C20008CEB93E062DF88E694E00E94801B88E9F9
:101C300094E0C5DE8EEC94E00E947F0188E994E098
:101C40003ADEFCCF4091A9055091AA0541155105F6
:101C500021F44091B3035091B4032091B503309126
:101C6000B6032115310549F48DB7282F30E0809156
:101C7000B1039091B203281B390B4217530718F098
:101C800080E090E00895C901841B950B089520E041
:101C900030E048EC52E40E9419300E94BB32DC0173
:101CA000CB010895AA2797FDA095BA2FBC01CD01BD
:101CB0000E94613220E030E048EC52E40C940E3196
:101CC0008F929F92AF92BF92CF92DF92EF92FF924C
:101CD0000F931F936C0154EEA52E54E0B52EC50151
:101CE000B60178D0882E0894C11CD11CC501B6015C
:101CF00071D0E82E0894C11CD11CC501B6016AD070
:101D0000982E0894C11CD11CC501B60163D090E087
:101D1000982F8827890D911DA0E0B0E0DC0199275C
:101D20008827FF24FE2CEE24E80CF11C00E010E0D4
:101D30008E0D9F1DA01FB11FBC01CD011F910F91E2
:101D4000FF90EF90DF90CF90BF90AF909F908F90DB
:101D50000895AF92BF92CF92DF92EF92FF920F93CE
:101D60001F938C016A017B01F4EEAF2EF4E0BF2ECD
:101D7000C501B8014C2D2AD00F5F1F4F5527F7FC26
:101D80005A954F2D3E2D2D2DC501B801422F1ED045
:101D90000F5F1F4F9701552737FD5095452FC50100
:101DA000B801422F13D00F5F1F4FCF2CDD24EE243C
:101DB000FF24C501B8014C2D09D01F910F91FF9050
:101DC000EF90DF90CF90BF90AF900895CB01642F3C
:101DD0000C947B3ACB010C94733A7093540160934A
:101DE0005301615070406230710530F081E090E045
:101DF000909354018093530108957093540160931C
:101E00005301615070406230710530F081E090E024
:101E1000909354018093530108958091490160E0AB
:101E20000E94F22D00008091490161E00E94F22D94
:101E30008AE090E00E94D72C8091490160E00E94E6
:101E4000F22D00000895EF92FF920F931F93CF930E
:101E5000DF937C018B010F701070C0914B01D0910A
:101E60004C0108C0602F61708C2F0E94F22D1595D7
:101E70000795219680915101909152018C179D07F1
:101E80008CF7C701CADFDF91CF911F910F91FF90AF
:101E9000EF900895EF92FF920F931F938C017B01B7
:101EA00094E0759567959A95E1F7C801CCDF8FE0CE
:101EB000E822FF24C801B701C6DF1F910F91FF90F0
:101EC000EF9008950F931F93CF93DF93EC018B0155
:101ED0008091450160E00E94F22D8091E50490918F
:101EE000E604892B29F08091470160E00E94F22DE1
:101EF000CE01B801A8DFDF91CF911F910F91089516
:101F00001F93CF93DF93EC01162F8091450161E081
:101F10000E94F22D8091E5049091E604892B29F02E
:101F20008091470160E00E94F22DE12FF0E0E49102
:101F30006E2F70E0CE01AEDFDF91CF911F9108953B
:101F4000EF92FF920F931F93CF93DF937C01042FA7
:101F5000EB0110E004C0C7016991D2DF1F5F1017C9
:101F6000D0F3DF91CF911F910F91FF90EF900895E3
:101F70000F931F93CF93DF93EC018B018091450169
:101F800061E00E94F22D8091E5049091E604892B96
:101F900029F08091470160E00E94F22DCE01B80146
:101FA00079DFDF91CF911F910F9108950F931F93C8
:101FB000CF93DF938C01EB0106C02196F901649168
:101FC00070E0C801D5DF9E01FE0184918823A9F746
:101FD000DF91CF911F910F91089564EE70E0E6CFED
:101FE000EF92FF921F93CF93DF937C01EB0110E000
:101FF00007C0AC0FBD1F6C9170E0C701B9DF1F5F58
:10200000A12FB0E0FE0101900020E9F73197EC1B11
:10201000FD0BAE17BF0768F3DF91CF911F91FF90C3
:10202000EF900895FB01E4916E2F70E0A1CF0F9324
:102030001F93CF93DF93EC018B018091450160E00A
:102040000E94F22D8091E5049091E604892B29F0FD
:102050008091470160E00E94F22DCE01B8011ADFA5
:10206000DF91CF911F910F910895EF92FF920F93FF
:102070001F938C017A0170E0DADFC801B70196DFA7
:102080001F910F91FF90EF900895CF93DF93EC0194
:102090008091490161E00E949F2D8091450161E09E
:1020A0000E949F2D8091E5049091E604892B29F0F0
:1020B0008091470161E00E949F2D80914B0161E07A
:1020C0000E949F2D80914D0161E00E949F2D809183
:1020D0004F0161E00E949F2D8091510161E00E94BB
:1020E0009F2D62E370E080E090E00E94B32CCE016F
:1020F00063E070E0E7DE65E070E080E090E00E9481
:10210000B32CCE0163E070E0DDDE84E690E00E9457
:10211000D72CCE0163E070E0D5DE65E070E080E0B2
:1021200090E00E94B32CCE0162E070E0CBDECE01E5
:1021300062E070E0C7DECE0168E070E0C3DE8CE3F1
:1021400090E00E94D72CCE016CE070E070DF8CE351
:1021500090E00E94D72CCE0161E070E068DF63E080
:1021600070E080E090E00E94B32CCE0166E070E069
:102170005EDF61E070E080E090E00E94B32CDF91D0
:10218000CF91089561E070E052DF61E070E080E09F
:1021900090E00C94B32C0895089581E08093F004AE
:1021A0006093EB041092EE041092EF040895F5CFC3
:1021B0008091EA049091E904891B08959091E904C3
:1021C0008091EA04981710F080E00895E091E70408
:1021D000F091E804E90FF11D80819F5F9093E9047D
:1021E00008959C018091F3049091F404892B11F1DE
:1021F0009091E9048091EA049817E0F090E00BC018
:10220000E091E704F091E804EA0FFB1FA20FB31F6F
:102210008C9180839F5FA92FB0E0A617B70784F346
:102220001092E9046093EA04E091F304F091F4045D
:10223000CB0109950895E091F104F091F2043097F3
:1022400029F01092EE041092EF040995089570930E
:10225000F4046093F30408957093F2046093F1041E
:1022600008950895DF93CF930F92CDB7DEB76983BA
:102270008091F0048823A9F08091EF048032A8F4C3
:102280008091EE04E091EC04F091ED04E80FF11D73
:1022900060838091EE048F5F8093EE048093EF045F
:1022A00004C0CE01019661E014D10F90CF91DF916F
:1022B0000895D8CFEF92FF920F931F93CF93DF93A0
:1022C0007C01042F8091F004882351F0EB0110E091
:1022D00004C0C7016991C6DF1F5F1017D0F303C0A8
:1022E000CB01642FF6D0DF91CF911F910F91FF901A
:1022F000EF900895FB0101900020E9F73197E61B6C
:10230000F70B4E2FD7CF6091EC047091ED048091C4
:10231000EB044091EF0421E097D01092EE0410926C
:10232000EF041092F0040895862F6091E7047091F5
:10233000E804413208F040E24FD01092E904809363
:10234000EA040895F1CF80E290E061E070E00E943D
:10235000D2369093E8048093E7041092E904109237
:10236000EA0480E290E061E070E00E94D23690934F
:10237000ED048093EC041092EE041092EF046AC214
:102380000F931F938C01862F23D08BE191E1C3D053
:1023900081EF90E1BBD0C801D6DF1F910F91089566
:1023A000EFCFFC0120E030E08081882311F421E0B0
:1023B00030E0C9010895FC0181E08083089508950B
:1023C0000895009711F00C94993708950C94EC3609
:1023D000880F8093BA000895982F413210F040E0A2
:1023E00031C08091F6048823E1F781E08093F60400
:1023F0008FEF809307051092FE0441504093FF0435
:102400004F5F990F91609093F70485EE8093BC0025
:102410008091F6048130E1F38091FE04841710F47A
:102420004091FE04A091FC04B091FD0420E030E056
:1024300007C0FB01E20FF31F8D9180832F5F3F4F99
:102440002417B8F3842F08951F93582F122F413269
:1024500010F081E03CC08091F6048823E1F782E02F
:102460008093F6048FEF809307051092FE0440934B
:10247000FF04A091FC04B091FD04FB0102C0819116
:102480008D938E2F861B8417D0F3852F90E0880FB5
:10249000991F8093F70485EE8093BC00112321F0EF
:1024A0008091F6048230E1F3809107058F3F11F4AB
:1024B00080E00DC080910705803211F482E007C0F2
:1024C00080910705803311F084E001C083E01F9103
:1024D0000895482F613210F081E008958091F6044C
:1024E000843011F082E0089560930305A091000507
:1024F000B0910105842F9C01F90102C081918D9357
:102500008E2F841B8617D0F380E008959093FB04F0
:102510008093FA0408959093F9048093F804089541
:10252000882311F085EC01C085E88093BC000895F4
:1025300085ED8093BC008091BC0084FDFCCF10929F
:10254000F604089585EC8093BC001092F60408957B
:102550001F920F920FB60F9211242F933F934F9318
:102560005F936F937F938F939F93AF93BF93EF93FB
:10257000FF938091B90090E0887F9070803691053C
:1025800009F4E2C081369105CCF58832910509F451
:102590007BC089329105B4F48031910509F46FC094
:1025A000813191053CF4009709F438C1089709F08E
:1025B00040C165C08831910509F466C0809709F073
:1025C00038C17FC08034910509F4A3C081349105DE
:1025D00044F48033910509F47FC0C89709F029C1FC
:1025E00086C08035910509F486C08835910509F4C7
:1025F00095C08834910509F01CC19EC088399105A9
:1026000009F404C189399105ECF48837910509F47E
:102610009BC0893791054CF48836910509F494C024
:102620008037910509F005C18FC08838910509F4FC
:10263000EDC08039910509F48DC08038910509F00D
:10264000F8C088C0803B910509F4B2C0813B910578
:102650004CF4803A910509F491C0883A910509F04B
:10266000E8C0A6C0803C910509F4D4C0883C91051F
:1026700009F4D0C0883B910509F0DBC0B1C080915E
:10268000F7048093BB00C0C09091FE048091FF04CA
:10269000981778F49091FE04E091FC04F091FD0409
:1026A000E90FF11D80818093BB009F5F9093FE0432
:1026B000ABC085ED8093BC008091BC0084FDFCCF55
:1026C000B6C080E28093070585ED8093BC008091C1
:1026D000BC0084FDFCCFABC080E38093070585ED93
:1026E0008093BC008091BC0084FDFCCFA0C088E337
:1026F000809307058FC08091FE049091BB00E0910C
:10270000FC04F091FD04E80FF11D90838F5F80932E
:10271000FE049091FE048091FF0474C08091FE0439
:102720009091BB00E091FC04F091FD04E80FF11DD5
:1027300090838F5F8093FE0485ED8093BC00809131
:10274000BC0084FDFCCF73C083E08093F60410923C
:1027500006055AC080910605803208F057C0809166
:1027600006059091BB00E0910405F0910505E80F86
:10277000F11D90838F5F8093060546C0809106050A
:10278000803248F480910605E0910405F09105053A
:10279000E80FF11D108260910605E091FA04F091B6
:1027A000FB04809104059091050570E0099532C005
:1027B00084E08093F6041092020510920305E091E4
:1027C000F804F091F904099580910305882341F4F8
:1027D00081E080930305E0910005F09101051082EE
:1027E00090910205E0910005F0910105E90FF11DBE
:1027F00080818093BB009F5F9093020590910205BA
:1028000080910305981710F485EC01C085E880934A
:10281000BC000FC085EC8093BC0009C01092070576
:1028200085ED8093BC008091BC0084FDFCCF1092AC
:10283000F604FF91EF91BF91AF919F918F917F919E
:102840006F915F914F913F912F910F900FBE0F901D
:102850001F9018951092F604449A459AE9EBF0E01F
:1028600080818E7F808380818D7F808388E48093C8
:10287000B80085E48093BC0080E290E061E070E005
:102880000E94D2368093FC049093FD0480E290E095
:1028900061E070E00E94D2368093000590930105BC
:1028A00080E290E061E070E00E94D23680930405FF
:1028B00090930505089508950895623018F080E01A
:1028C00090E00895E62FF0E03196EE0FFF1FE80F3D
:1028D000F91F808191810895FC01662309F4148217
:1028E00008950F931F93CF93DF93EC018A0167FF45
:1028F00004C070E0888199819ADB88819981B80150
:102900006FDBDF91CF911F910F910895FF920F938D
:102910001F93CF93DF93EC01262F277019F43EEF1E
:10292000F32E01C0F22E862F90E0821B910968E001
:1029300070E00E94A235623009F460C0633030F468
:10294000662359F0613009F0ACC035C0633009F43A
:102950006DC0643009F0A5C076C0042F10E00058A7
:102960001F4F88819981B80162DB888199816EEF60
:1029700070E0FEDA005C1F4F88819981B80157DB57
:10298000888199816EEF70E0F3DA0C5210408881F3
:102990009981B8014CDB888199816EEF70E0E8DAAB
:1029A000005C1F4F88819981B80141DB6F2D70E079
:1029B0008881998175C0042F10E000581F4F8881CD
:1029C0009981B80134DB888199816EEF70E0D0DAAB
:1029D000005C1F4F88819981B80129DB888199812A
:1029E0006EEF70E0C5DA0C52104088819981B80111
:1029F0001EDB6F2D70E08881998147C0042F10E0A5
:102A000000581F4F88819981B80111DB8881998115
:102A10006EEF70E0ADDA005C1F4F88819981B801DC
:102A200006DB6F2D70E08881998124C0042F10E0AF
:102A300000581F4F88819981B801F9DA6F2D70E035
:102A4000888199810CC0042F10E000581F4F8881A5
:102A50009981B801ECDA888199816FEF70E088DAAA
:102A6000005C1F4F88819981B801E1DA88819981E2
:102A70006FEF70E07DDA0C52104088819981B801C7
:102A8000D6DA888199816FEF70E072DA005C1F4FAF
:102A900088819981B801CBDA888199816FEF70E0E4
:102AA00067DADF91CF911F910F91FF900895EF9218
:102AB000FF921F93CF93DF937C01EC0110E0C701DD
:102AC0006E81412F23DF888599859F838E8322968F
:102AD0001F5F1331A1F7DF91CF911F91FF90EF900E
:102AE0000895DF92EF92FF920F931F93CF93DF939E
:102AF000EC01D62E842F6AE00E949635082F282FED
:102B000030E086EF9FEFBC01269FC001279F900D0C
:102B1000369F900D1124840F911D62E070E00E9499
:102B2000A2357B0110E017C0101728F48881998125
:102B30006FEF70E008C0101741F488819981E114AB
:102B4000F10429F0B70114DA05C08881998165E59F
:102B500071E046DA1F5F1D1538F3DF91CF911F91A9
:102B60000F91FF90EF90DF900895CF92DF92EF9258
:102B7000FF920F931F93CF93DF938C016A01660F2F
:102B8000660F660FC0E0D0E06064E62EFF24BE0151
:102B90006E297F29F8018081918149DAF601EC0FD5
:102BA000FD1F608170E0F80180819181E1D921965B
:102BB000C830D10561F7DF91CF911F910F91FF9040
:102BC000EF90DF90CF900895CF92DF92EF92FF9237
:102BD0000F931F93CF93DF938C016A01660F660FEB
:102BE000660FC0E0D0E06064E62EFF24BE016E29CF
:102BF0007F29F801808191811ADAF601EC0FFD1F1F
:102C0000E4916E2F70E0F80180819181B1D9219615
:102C1000C830D10559F7DF91CF911F910F91FF90E7
:102C2000EF90DF90CF9008950F931F938C0161E098
:102C300041ED51E0C9DFC80162E049ED51E0C4DF78
:102C4000C80163E041EE51E0BFDFC80164E049EE36
:102C500051E0BADFC80165E041EF51E0B5DFC801DE
:102C600066E049EF51E0B0DFC80167E041E052E0C3
:102C7000ABDF1F910F9108950F931F938C0161E0BB
:102C800041EB51E0A1DFC80162E049EB51E09CDF7C
:102C9000C80163E041EC51E097DFC80164E049EC12
:102CA00051E092DF1F910F9108950F931F938C01B4
:102CB00065E041E951E088DFC80166E049E951E09B
:102CC00083DFC80167E041EA51E07EDFC80168E0C8
:102CD00049EA51E079DF1F910F9108950F931F93F7
:102CE0008C0165E041E751E06FDFC80166E049E72C
:102CF00051E06ADFC80167E041E851E065DFC801E3
:102D000068E049E851E060DF1F910F9108950F934B
:102D10001F938C0161E041E551E056DFC80162E09C
:102D200049E551E051DFC80163E041E651E04CDF85
:102D3000C80164E049E651E047DF1F910F91089513
:102D40000F931F938C0161E041E151E03DDFC80129
:102D500062E049E151E038DFC80163E041E251E05F
:102D600033DFC80164E049E251E02EDFC80165E0CD
:102D700041E351E029DFC80166E049E351E024DF87
:102D8000C80167E041E451E01FDFC80168E049E4A1
:102D900051E01ADF1F910F9108950F931F938C013B
:102DA00061E049EE50E010DFC80162E041EF50E021
:102DB0000BDFC80163E049EF50E006DFC80166E0C1
:102DC00041E051E001DFC80168E049E051E0FCDE8C
:102DD0001F910F9108950F931F93CF93DF93EC01F1
:102DE000062F10E006C0888199816EEF70E0C0D890
:102DF0001F5F1017C0F3DF91CF911F910F910895BE
:102E0000FF920F931F93CF93DF93EC01162FCA010C
:102E1000F22E6EA57FA54AE050E00E94E239AEA5F1
:102E2000BFA5FD0101900020E9F73197EA1BFB0BDC
:102E30000F2D0E1BCE01612FAD0153DD002329F0B4
:102E4000FF2019F0CE01602FC6DFDF91CF911F91D7
:102E50000F91FF9008956F927F928F929F92AF9201
:102E6000BF92CF92DF92EF92FF920F931F93CF9377
:102E7000DF937C01A62EC42EDD2459E5652E51E09A
:102E8000752E620E711CF3018081B601680F711DF1
:102E9000F70180819181CBD8CA2DD0E05E01AA0CC8
:102EA000BB1CAA0CBB1C0DEA11E0F801EA0DFB1DCE
:102EB000608170E0F701808191815AD845010894C2
:102EC000811C911CF801E80DF91D608170E0F7018B
:102ED000808191814DD8E50122960C0F1D1FF801CC
:102EE000608170E0F7018081918142D8F301818196
:102EF000B601680F711DF7018081918198D805EDA9
:102F000011E0F801EA0DFB1D608170E0F70180819E
:102F100091812ED8F801E80DF91D608170E0F7016C
:102F20008081918125D80C0F1D1FF801608170E010
:102F3000F701808191811CD8F3018281B601680F6D
:102F4000711DF7018081918172D80DEF11E0F801B8
:102F5000EA0DFB1D608170E0F7018081918108D846
:102F6000F801E80DF91D608170E0F7018081918121
:102F70000E94B80F0C0F1D1FF801608170E0F7016F
:102F8000808191810E94B80FF3018381C80ED11C0A
:102F9000F70180819181B6014AD805E212E0A00EC6
:102FA000B11EF501608170E0F701808191810E947E
:102FB000B80F800E911EF401608170E0F7018081EE
:102FC00091810E94B80F0C0F1D1FF801608170E005
:102FD000F701808191810E94B80FDF91CF911F91FD
:102FE0000F91FF90EF90DF90CF90BF90AF909F90A8
:102FF0008F907F906F9008952F923F924F925F92A3
:103000006F927F928F929F92AF92BF92CF92DF92F8
:10301000EF92FF920F931F935C01E62E642E7724AC
:10302000F9E52F2EF1E03F2E220E311CF1018081B7
:10303000B301680F711DF501808191810E94171005
:10304000FF242701440C551C440C551C7DE5C72E5C
:1030500071E0D72EF601E40DF51D608170E0F501F9
:10306000808191810E94B80F8701000F111F0E0D02
:103070001F1D0894E11CF11C4701800E911EF601F2
:10308000E80DF91D608170E0F501808191810E9459
:10309000B80F0894E11CF11CE00EF11ECE0CDF1CF1
:1030A000F601608170E0F501808191810E94B80F86
:1030B000F1018181680E711CF50180819181B3015C
:1030C0000E94171005E811E0400E511EF2016081C8
:1030D00070E0F501808191810E94B80F800E911EF1
:1030E000F401608170E0F501808191810E94B80F48
:1030F0000E0D1F1DF801608170E0F5018081918146
:103100000E94B80F1F910F91FF90EF90DF90CF902A
:10311000BF90AF909F908F907F906F905F904F90F7
:103120003F902F9008952F923F924F925F926F920F
:103130007F928F929F92AF92BF92CF92DF92EF9247
:10314000FF920F931F93DF93CF93CDB7DEB76A97AC
:103150000FB6F894DEBF0FBECDBF6C015B01642ECD
:10316000922E402E5E2C822F840F888F1A8293E637
:103170009A8F198E7724882410E01E010894211C50
:10318000311CB3E0EB2EF12CEC0EFD1E28C0AA0D75
:10319000BB1D8C918983112339F48D3229F47394EA
:1031A0008394E1E0E98F0DC08E3221F08B3311F072
:1031B0008C3239F4F701E10FF11D808373941A8F7B
:1031C0000DC080538A3050F4C1010E940F39F701BD
:1031D000E10FF11D80837394F4E08F0E1F5FA12F28
:1031E000B0E0F50101900020E9F73197EA19FB09F9
:1031F000AE17BF0760F2862D90E088199109181666
:10320000190624F5842D90E0A9E5EA2EA1E0FA2E16
:10321000E80EF91E8C01050D111D075A1E4FA92C31
:10322000BB24962C97180EC0F70181917F01B50140
:10323000680F711DF601808191810E941710C601EF
:10324000692DC9DDE016F10679F76AC010E0F88D46
:103250002F2E3324E42CFF2489E591E0E80EF91E9B
:1032600057010894A11CB11C57C01123E9F4998D92
:103270009923D1F0F60120813181692D70E0F4E0CD
:103280005F1611F4F50101C0F7018081680F711D0F
:10329000C9010E941710F6018081918168E070E0F9
:1032A0000E94B80F939437C0FA8D1F1781F4F6016E
:1032B00020813181F4E05F1621F4C9016FEF70E0E5
:1032C00003C0C90165E070E00E94B80F24C0892DD9
:1032D00090E0039682159305F4F4E12FF0E082E08C
:1032E000581661F483E090E08C0F9D1FE80FF91FE2
:1032F000C6016081492D242D7FDE0BC083E090E064
:103300008C0F9D1FE80FF91FC6016081492D242DE8
:10331000A2DD94E0990E1F5F171508F4A6CF03C035
:10332000988C981893CF6A960FB6F894DEBF0FBEAC
:10333000CDBFCF91DF911F910F91FF90EF90DF9064
:10334000CF90BF90AF909F908F907F906F905F9045
:103350004F903F902F900895CF92DF92EF92FF927F
:103360000F931F936C01CB01142FF22EF60166A56B
:1033700077A54AE050E00E94E239F60166A577A5FC
:10338000C601412F2F2DCFDE1F910F91FF90EF909F
:10339000DF90CF900895FC01633008F062E0658310
:1033A000E62FF0E0EA51FF4F6591749185E00C94AF
:1033B000412DFC018581833011F4158202C08F5F9D
:1033C0008583CF016581E7CFCF92DF92EF92FF92A5
:1033D0000F931F938C016B019ADCC8017FDCC8013D
:1033E00062E0D9DF83E06FEF70E00E94412D62E37D
:1033F00070E080E090E00E94B32C83E068E270E02F
:103400000E94412D62E370E080E090E00E94B32CC6
:1034100083E060E070E00E94412DEE24D7FCE09450
:10342000FE2CC701B6010E94B32C1F910F91FF9093
:10343000EF90DF90CF9008956F927F928F929F923E
:10344000AF92BF92CF92DF92EF92FF920F931F93B2
:10345000DF93CF93CDB7DEB76E970FB6F894DEBF8C
:103460000FBECDBF3B0169017A014801CA01B90114
:1034700020E030E040E050E00E940B3288232CF046
:10348000C701B6010E94563604C0C701B6010E94AA
:1034900043360E94BB325B01B501882777FD8095DA
:1034A000982F0E9461329B01AC01C701B6010E94B6
:1034B000C72F7B018C01B401882777FD8095982F59
:1034C0000E9461329B01AC01C801B7010E94193012
:1034D0000E94BB326B0177FF09C0D094C194D10820
:1034E000D394A114B10411F441E001C040E0C4013F
:1034F0006AE070E00E94A2357B0199242AE030E066
:103500000EC0C216D3060CF49394C901880F991FFC
:1035100013E0220F331F1A95E1F7280F391FE21627
:10352000F3067CF7442381F08DE28983C501BE0157
:103530006E5F7F4F4AE050E00E94E2399E01205FBB
:103540003F4FF90190E306C0C501BE016F5F7F4F99
:10355000F1CF91938E2F821B8915D8F38E01005FD6
:103560001F4FB801690D711DC6014AE050E00E946D
:10357000E239E00EF11EF7011082C301BE016F5F58
:103580007F4F0E949939C30167E571E00E947A3943
:10359000C301B8010E947A396E960FB6F894DEBF67
:1035A0000FBECDBFCF91DF911F910F91FF90EF9094
:1035B000DF90CF90BF90AF909F908F907F906F9053
:1035C00008956F927F928F929F92AF92BF92CF9207
:1035D000DF92EF92FF920F931F935C013A014B0130
:1035E000F22ED02EFC0166A577A5A401930104E676
:1035F00010E022DFF50166A577A5C5014F2D2D2D21
:103600000E2DEC2C90DD1F910F91FF90EF90DF902D
:10361000CF90BF90AF909F908F907F906F900895C4
:10362000AF92BF92CF92DF92EF92FF920F931F93D0
:103630007C015A016B018901FC0166A577A5A601F1
:103640009501FADEF70166A577A5808191810E9438
:10365000F00F1F910F91FF90EF90DF90CF90BF90F0
:10366000AF900895AF92BF92CF92DF92EF92FF9208
:103670000F931F935C0169017A0170E0FC01808166
:1036800091810E941710C501B701A6019801C8DFFA
:103690001F910F91FF90EF90DF90CF90BF90AF9070
:1036A00008950F931F9304E610E0DCDF1F910F9144
:1036B000089524E630E0B4CFDC011496EC91149721
:1036C000F0E03196EE0FFF1FEA0FFB1F8081918122
:1036D000B2C0DC011496EC911497F0E03196EE0F35
:1036E000FF1FEA0FFB1F80819181C0C0FC01848114
:1036F000882311F4148202C08F5F8483CF01E9CF45
:103700000F931F93CF93DF93EC011C8282E08D8394
:1037100081E090E00E94E6118C0164E070E00E947C
:10372000FD0E1983088385E190E00E94EC369FA787
:103730008EA7888199810E944510FE0180E090E06B
:10374000178216820196329684319105C9F789E075
:1037500090E00E94E6118C0196D11B830A83DF91D1
:10376000CF911F910F910895FC0181E592E0918323
:10377000808380916804909169049383828314828A
:103780001582168217820895FC0181E592E09183EB
:10379000808380916804909169049383828314826A
:1037A0001582168217820895FC0181E592E09183CB
:1037B00080837383628360E070E044835583668313
:1037C00077830895FC0181E592E091838083738380
:1037D000628360E070E04483558366837783089555
:1037E000FC018481982F937E8C71843011F4986051
:1037F00001C0946094830895FC012581922F9295D5
:103800009F703681832F8295807F892B865F982FCA
:103810009295907F2F70292B2583982F92959F70DA
:10382000307F392B36838E3620F02F702583307F02
:10383000368310860895CF93DF93EC0128859D8110
:1038400092959F708E818295807F892B281749F4ED
:10385000E881F9810280F381E02DCE010995188677
:1038600002C02F5F2887DF91CF910895CF93DF9318
:10387000EC018A819B810E9445108C8187FF03C0E7
:1038800088E694E0F9D98D8181FF03C088E694E051
:10389000CBD98D8180FF03C088E694E006DA8D8164
:1038A00083FF03C088E694E078DA8D8182FF03C04D
:1038B00088E694E045DA8C818170809399048C814C
:1038C0008695817080939A048C8182958695837009
:1038D000809398049D8192959F708E818295807FC0
:1038E000892B8887E881F9810190F081E02DCE0154
:1038F0000995DF91CF910895FC0189E592E09183CC
:1039000080830895FC0189E592E091838083089586
:10391000EF92FF921F93FC018281938165E870E032
:103920000E94171088E6E82E84E0F82E40910E04DD
:1039300050910F04C70165E823E062DA209110047A
:10394000309111044091120450911304C7016EE8A4
:10395000A8DE60915A01685F209106043091070447
:103960004091080450910904C7019BDE60915B01FE
:103970006B5F40910C0450910D04C70124E040DAC4
:1039800060915B01625F2091FE033091FF034091E3
:10399000000450910104C70184DE10915C018FE0A6
:1039A0000E94262EAC01C701612F21E029DA109177
:1039B0005C011B5F6091E20470E080E090E00E9497
:1039C0000C339B01AC01C701612F6BDE10915C01D0
:1039D000175F6091E30470E080E090E00E940C3398
:1039E0009B01AC01C701612F5CDE60915C01635FEC
:1039F0002091D9043091DA044091DB045091DC0429
:103A0000C7014FDE1F91FF90EF9008950F931F9312
:103A10008C01FC0182819381609159014FE152E058
:103A20000E94351060915901665FF801828193818F
:103A30004BE152E00E943510F80182819381609140
:103A40005A0143E152E00E943510F80182819381CE
:103A500060915B014EE052E00E94351060915B0185
:103A6000665FF8018281938149E052E00E9435103F
:103A70001F910F910895FC0189E592E09183808365
:103A8000CF010C94E1110F931F938C016DDE89E53A
:103A900092E0F8019183808394819C718681807F7C
:103AA00086839364948384EA85831F910F9108959C
:103AB0000F931F938C0158DE89E592E0F801918302
:103AC000808394819C718681807F868393649483B4
:103AD00084EA85831F910F910895FC011486138653
:103AE00088E893E1928781870895FC018481282FDB
:103AF000269526952F5F2770922F990F990F837E19
:103B0000892B848330E0263031051CF0837E84606D
:103B100084830895AF92BF92CF92DF92EF92FF928B
:103B20000F931F93CF93DF93EC018C81869586953D
:103B3000877090E08330910539F18430910534F439
:103B40008130910559F0029731F412C0843091050B
:103B500051F00597F1F020E030E01FC02091BE0346
:103B60003091BF031AC020910E0430910F0415C08C
:103B700060911404709115048091160490911704BB
:103B80000E94BB329B0109C020910C0430910D04AE
:103B900004C020910A0430910B0489859A85281766
:103BA000390714F43A8729878B859C8582179307F8
:103BB00014F43C872B8700D000D0B901882777FD0B
:103BC0008095982F29853A85442737FD4095542FB5
:103BD000EB84FC840027F7FC0095102FE1E2AE2E69
:103BE000B12CC12CD12CEDB7FEB7A182B282C38219
:103BF000D482AA24BB246501D6D50F900F900F90D4
:103C00000F906132710514F060E270E08B0177FF74
:103C100002C000E010E088E694E0602F43E10E94DB
:103C20008614109395040093940488E694E00E940F
:103C300057154C8146954695477050E088E694E0CC
:103C400060E820E0DDD88A819B8161E672E00E9415
:103C5000F00F488550E088E694E060E020E0D0D89E
:103C60004091A0045091A1046091A2047091A3041A
:103C70008CE895E02AE030E063D4DF91CF911F918A
:103C80000F91FF90EF90DF90CF90BF90AF9008958D
:103C90000F931F938C0168DD87E692E0F801918312
:103CA000808395818681807F868384E08483987079
:103CB000926A95831F910F9108950F931F938C0122
:103CC00053DD87E692E0F8019183808395818681B8
:103CD000807F868384E084839870926A95831F91A5
:103CE0000F910895FC0181858F5F8187843008F0F2
:103CF00011860895CF93DF93EC01498550E088E663
:103D000094E064E820E07CD88A819B8163EC70E0D9
:103D10000E941710E985F0E0EE0FFF1FEE0FFF1F66
:103D2000E05DFB4F608171818281938120E030E012
:103D300040E050E00E9436322A813B81882324F4FF
:103D4000C9016BE672E003C0C9016DE672E00E9432
:103D5000F00FE985F0E0EE0FFF1FEE0FFF1FE05DB3
:103D6000FB4F60817181828193810E94BB329B01F4
:103D700077FF03C0309521953F4FB901882777FD24
:103D80008095982F0E946132AB01BC0188E694E0D7
:103D900090DCE985F0E0EE0FFF1FEE0FFF1FE05C07
:103DA000FB4F4081518188E694E06EEC20E028D8FA
:103DB000E985F0E0EE0FFF1FEE0FFF1FE05BFB4F0A
:103DC00060817181828193810E94BB329B01AC0131
:103DD00088E694E068E9A90120E012D8E985F0E0DE
:103DE000EE0FFF1FE85DFB4F4081518188E694E0B4
:103DF00062EA20E005D8DF91CF9108950F931F93D9
:103E00008C01FC018281938160E842E452E00E94CF
:103E10003510F8018281938160EC43E352E00E9407
:103E20003510F8018281938164E944E252E00E94F6
:103E300035101F910F9108950F931F938C0194DCFF
:103E400083E792E0F8019183808394819C712581BE
:103E500028708681807F8683936494832062258383
:103E600011861F910F9108950F931F938C017CDC95
:103E700083E792E0F8019183808394819C7125818E
:103E800028708681807F8683936494832062258353
:103E900011861F910F9108951F920F920FB60F92E6
:103EA00011242F933F934F938F939F93EF93FF93FF
:103EB0004091C600E0918805F091890531969F01F7
:103EC0002F773070319780918A0590918B05281754
:103ED000390739F0E85FFA4F408330938905209322
:103EE0008805FF91EF919F918F914F913F912F9175
:103EF0000F900FBE0F901F9018958F92AF92CF9298
:103F0000DF92EF92FF920F931F93DF93CF93CDB782
:103F1000DEB7FC018BE792E0918380837383628339
:103F2000558344833783268311870087F386E2868F
:103F3000D586C486A68687868D85808B8E85818B67
:103F40008F85828BCF91DF911F910F91FF90EF9022
:103F5000DF90CF90AF908F9008958F92AF92CF92D5
:103F6000DF92EF92FF920F931F93DF93CF93CDB722
:103F7000DEB7FC018BE792E09183808373836283D9
:103F8000558344833783268311870087F386E2862F
:103F9000D586C486A68687868D85808B8E85818B07
:103FA0008F85828BCF91DF911F910F91FF90EF90C2
:103FB000DF90CF90AF908F900895CF93DF93EC0177
:103FC0009A01AB01E885F985203081EE380780E061
:103FD000480780E0580709F445C081E090E00A886E
:103FE00002C0880F991F0A94E2F7808360E079E0AD
:103FF0008DE390E00E94B535215030404040504064
:104000005695479537952795EC81FD813083EE8154
:10401000FF812083EA85FB85208141E050E0CA01D1
:104020000E8402C0880F991F0A94E2F7282B208380
:10403000EA85FB852081CA010F8402C0880F991F81
:104040000A94E2F7282B2083EA85FB858081088883
:1040500002C0440F551F0A94E2F7842B8083DF913E
:10406000CF910895108220E130E0CECFFC01A285EF
:10407000B3854C9121E030E0C901068402C0880F6D
:10408000991F0A94E2F7809584238C93A285B385C7
:104090004C91C901078402C0880F991F0A94E2F766
:1040A000809584238C93A285B3858C91008802C06F
:1040B000220F331F0A94E2F7209528232C930895AA
:1040C000DC011296ED91FC911397E058FF4F21917E
:1040D000319180819181281B390B2F773070C90174
:1040E0000895DC011296ED91FC911397EE57FF4F66
:1040F0002081318192918291E058F040821793079C
:1041000019F42FEF3FEF05C0E20FF31F8081282F36
:1041100030E0C9010895DC011296ED91FC911397EE
:10412000DF01AE57BF4F2D913C911197E058FF4FE3
:1041300080819181E058F0408217930719F42FEFA6
:104140003FEF0BC0E20FF31F80812F5F3F4F2F77B0
:1041500030702D933C93282F30E0C9010895DC0185
:104160001296ED91FC911397EE57FF4F808191814C
:10417000929382930895FC01A085B18521898C9149
:1041800090E0022E02C0959587950A94E2F780FF91
:10419000F6CF0484F585E02D608308958BE792E0E7
:1041A00090938D0580938C0588E095E090938F0522
:1041B00080938E0585EC90E0909391058093900517
:1041C00084EC90E0909393058093920580EC90E0CE
:1041D000909395058093940581EC90E090939705DA
:1041E0008093960586EC90E09093990580939805CE
:1041F00084E080939A0583E080939B0587E0809319
:104200009C0585E080939D0581E080939E0508953F
:104210000F931F93CF93DF938C01EB0109C021967D
:10422000D801ED91FC910190F081E02DC801099534
:1042300068816623A1F7DF91CF911F910F910895B7
:10424000EF92FF920F931F93CF93DF938C017B012B
:10425000EA010CC0D7016D917D01D801ED91FC916F
:104260000190F081E02DC80109952197209791F7E1
:10427000DF91CF911F910F91FF90EF900895DC0196
:10428000ED91FC910280F381E02D09950895CF9284
:10429000DF92EF92FF920F931F93CF93DF936C0106
:1042A0007B01C0E0D0E00DC0D601ED91FC91008112
:1042B0001181C701BE013DD3682FC601F8010995E0
:1042C0002196F70184819581C817D90768F3DF919A
:1042D000CF911F910F91FF90EF90DF90CF900895B5
:1042E0002F923F924F925F926F927F928F929F9206
:1042F000AF92BF92CF92DF92EF92FF920F931F93F4
:10430000DF93CF93CDB7DEB7A0970FB6F894DEBF9B
:104310000FBECDBF1C016A017B014115510561052E
:10432000710541F440E350E060E070E020E030E0EF
:104330009BD053C0882499245401422E55246624CE
:10434000772401E010E00C0F1D1F080D191DC70197
:10435000B601A30192010E94B535F801608308946B
:10436000811C911CA11CB11CC701B601A3019201C3
:104370000E94B535C901DA016C017D01C114D10477
:10438000E104F104F1F681E0E82EF12CEC0EFD1EC3
:10439000E80CF91C3E010894611C711CD501C40194
:1043A0000197A109B1096C01C818D90813C0F60119
:1043B000EE0DFF1D40814A3010F4405D01C0495CA4
:1043C00050E060E070E0C10120E030E04DD00894A2
:1043D000E108F1086E147F0451F7A0960FB6F89427
:1043E000DEBF0FBECDBFCF91DF911F910F91FF9028
:1043F000EF90DF90CF90BF90AF909F908F907F9085
:104400006F905F904F903F902F900895DC012115A1
:10441000310541F4ED91FC910190F081E02D642F84
:10442000099508955DCFEF92FF920F931F939A0124
:104430007B0100E010E0B801A701E8DF1F910F91B8
:10444000FF90EF900895EF92FF920F931F939A01C0
:10445000E62EFF2400E010E0B801A701D7DF1F918E
:104460000F91FF90EF900895EF92FF920F931F939B
:10447000CF93DF93EC017A018B012115310541F4D3
:10448000E881F9810190F081E02D642F099519C030
:104490002A303105A9F477FF0FC04DE250E060E00B
:1044A00070E020E030E0E0DF10950095F094E094BB
:1044B000E11CF11C011D111DCE01B801A7012AE06C
:1044C0000FDFDF91CF911F910F91FF90EF90089533
:1044D000EF92FF920F931F937B019A010027F7FC45
:1044E0000095102FB801A701BFDF1F910F91FF901A
:1044F000EF900895EF92FF920F931F939A01E62E8B
:10450000FF2400E010E0B801A701AEDF1F910F917A
:10451000FF90EF9008950F931F938C014DE050E0B2
:1045200060E070E020E030E09FDFC8014AE050E04A
:1045300060E070E020E030E097DF1F910F91089578
:104540000F931F938C0162DFC801E5DF1F910F916C
:104550000895CF92DF92EF92FF920F931F938C01F9
:104560009A016B01EE24FF24B701A6014FDFC801B9
:10457000D2DF1F910F91FF90EF90DF90CF900895C1
:10458000CF92DF92EF92FF920F931F938C019A01CB
:10459000C62EDD24EE24FF24B701A60137DFC801B3
:1045A000BADF1F910F91FF90EF90DF90CF900895A9
:1045B0000F931F938C0163DEC801ADDF1F910F9134
:1045C00008950F931F93CF93DF938C01EB010AC0E3
:1045D0002196F901449150E060E070E0C80120E0CC
:1045E00030E014DF9E01FE018491882389F7C80121
:1045F00092DFDF91CF911F910F9108950F931F9339
:104600008C0145DEC80187DF1F910F9108950F933C
:104610001F938C0129DFC8017EDF1F910F91089540
:10462000CF92DF92EF92FF920F931F938C016B0159
:104630009A01EE24D7FCE094FE2CB701A60114DF0A
:10464000C80169DF1F910F91FF90EF90DF90CF902D
:104650000895CF92DF92EF92FF920F931F938C01F8
:104660009A01C62EDD24EE24FF24B701A601FCDE4C
:10467000C80151DF1F910F91FF90EF90DF90CF9015
:1046800008959F92AF92BF92CF92DF92EF92FF92E6
:104690000F931F93CF93DF93EC017A018B01922E3E
:1046A000CB01BA0120E030E040E050E00E94363219
:1046B000882364F4CE014DE250E060E070E020E039
:1046C00030E0D2DE17FB109517F9109520E030E0AE
:1046D00040E05FE3AA240BC0CA01B90120E030E04A
:1046E00040E251E40E940E319B01AC01A394A91455
:1046F00098F3C801B7010E94F22F5B016C010E9480
:10470000552E7B018C01CE01B801A7012AE030E0D3
:104710007DDE992021F0CE016BE972E0B0DDC801A9
:10472000B7010E940C339B01AC01C601B5010E9488
:10473000C72F21C020E030E040E251E40E94193050
:104740007B018C010E94BB325B016C01CC24B7FC65
:10475000C094DC2CCE01B601A5012AE030E084DE55
:10476000C601B5010E9461329B01AC01C801B701CD
:104770000E94C72F9A949920E9F6DF91CF911F915B
:104780000F91FF90EF90DF90CF90BF90AF909F90F0
:10479000089577CF0F931F938C0173DFC801BBDEA1
:1047A0001F910F9108952F923F924F925F926F92B7
:1047B0007F928F929F92AF92BF92CF92DF92EF92B1
:1047C000FF920F931F93DF93CF93CDB7DEB73B01DB
:1047D0004C0119012A016D897E898F89988D6A198A
:1047E0007B098C099D09621A730A840A950AA4013F
:1047F00093010E947735E218F30804091509A8010E
:1048000097010E94D7352A0D3B1D4C1D5D1DB90136
:10481000CA01CF91DF911F910F91FF90EF90DF9030
:10482000CF90BF90AF909F908F907F906F905F9050
:104830004F903F902F900895089570E0382F20E01A
:10484000622B732BCB010895EF92FF920F931F936E
:104850007B018C01611571058105910529F420E02A
:1048600030E040E050E00BC00E943C38A8019701C6
:104870000E94D735AC01CB01DA019C01AD01B90131
:10488000CA011F910F91FF90EF900895EF92FF9250
:104890000F931F937B018C016217730784079507A1
:1048A0005CF4261B370B480B590BCA01B901CCDF4E
:1048B000E60EF71E081F191FB701C8011F910F91BF
:1048C000FF90EF900895009729F0BC0180E090E000
:1048D0000C943F380895FC010190F081E02DE60F23
:1048E000F71F80810895DC01ED91FC9111973097BD
:1048F00051F014968D919C9115976817790718F4CB
:10490000E60FF71F40830895FC019B018481958188
:104910006817790728F4608171816115710529F4A0
:1049200010929F056FE975E002C0620F731FCB0103
:104930000895FC010190F081E02DE60FF71F8081C2
:104940000895FC01808191810C942C390F931F9361
:10495000CF93DF93FC018B0141155105A1F0611547
:10496000710589F084819581EA0121978C179D0753
:1049700008F4EC0160817181C801AE010E94AE397A
:10498000C00FD11F1882DF91CF911F910F91089511
:104990000F931F93CF93DF93FC018B0141155105BA
:1049A000A1F06115710589F084819581EA01219753
:1049B0008C179D0708F4EC0160817181C801AE017C
:1049C0000E94AE39C00FD11F1882DF91CF911F9185
:1049D0000F9108950F931F938C01FC0180819181A9
:1049E0000E949937F80113821282158214821F9156
:1049F0000F910895FC01DB0114962D913C911597C0
:104A000084819581821B930B8417950710F480E0B5
:104A10000895808191816D917C91840F951FA901EA
:104A20000E94A0399C0180E0232B09F481E00895C5
:104A3000FC01DB012481358114968D919C911597A1
:104A40002817390710F480E00895CF0140E050E0C6
:104A5000D1CFDF92EF92FF920F931F93CF93DF930B
:104A6000EC018C819D8148175907B8F47A010894AC
:104A7000E11CF11CE881F981EE0DFF1DD080108250
:104A800008811981C80170E00E94BD399C010E0D9A
:104A90001F1DF801D082009719F4EFEFFFEF05C05A
:104AA00088819981F901E81BF90BCF01DF91CF9142
:104AB0001F910F91FF90EF90DF900895FC014481CA
:104AC000558141505040C5CFCF93DF93FC01DB01AE
:104AD000848195814817590760F4C081D1816D9117
:104AE0007C91CE01840F951F0E94C8399C010097CC
:104AF00019F42FEF3FEF02C02C1B3D0BC901DF91D2
:104B0000CF91089540E050E0DFCFCF93DF93FC01D9
:104B1000848195814817590758F4C081D181CE010D
:104B2000840F951F70E00E9485399C01009719F44D
:104B30002FEF3FEF02C02C1B3D0BC901DF91CF913E
:104B4000089540E050E0E1CFDC01FB0114962D9187
:104B50003C911597848195812817390711F080E0E1
:104B60000895608171818D919C910E9490399C0182
:104B700080E0232B09F481E00895FC01DB0124810E
:104B8000358114968D919C9115972817390710F44B
:104B900080E00895281B390B808191816D917C9173
:104BA000820F931F0E9490399C0180E0232B09F40F
:104BB00081E00895DC01FB01608171818D919C9100
:104BC0000E949039292F332727FD30952095309565
:104BD0002227330F221F3327C9010895DC01FB016F
:104BE000608171818D919C910E94903940E050E0EC
:104BF0001816190614F041E050E0CA010895DC01CE
:104C0000FB01608171818D919C910E94903940E0FF
:104C100050E01816190614F441E050E0CA01089556
:104C2000DC01FB01608171818D919C910E94903922
:104C3000292F332727FD30952227330F221F3327B3
:104C4000C9010895DC01FB0114962D913C91159743
:104C5000848195812817390751F4608171818D9184
:104C60009C910E9490399C0180E0232B09F081E007
:104C700090E00895DC01FB0114962D913C9115976D
:104C8000848195812817390711F080E00BC060817D
:104C900071818D919C910E9490399C0180E0232B21
:104CA00009F481E090E00895FC01DB016D917C91B5
:104CB000808191810C9490390F931F93CF93DF9350
:104CC000EC018B01FB01648175818C819D81680FF2
:104CD000791F7D836C838A819B8186179707B8F43F
:104CE0006F5F7F4F888199810E9448384C815D8138
:104CF000009729F0998388835B834A8308C0F80171
:104D000084819581481B590B5D834C8307C0F80152
:104D100060817181888199810E947A39CE01DF9109
:104D2000CF911F910F910895C7CFCF93DF93EC01DF
:104D3000CB017B836A8301960E94EC36998388833A
:104D4000009721F41B821A821D821C82DF91CF9171
:104D500008950F931F93CF93DF93EC018B01861778
:104D6000970701F1FB01248135818C819D81821798
:104D7000930748F4888199810E949937F8016481EA
:104D80007581CE01D2DF288139812115310551F09D
:104D9000F801848195819D838C8360817181C90133
:104DA0000E949939CE01DF91CF911F910F91089503
:104DB0001F93CF93DF93EC01162F81E090E09D834A
:104DC0008C83CE0161E070E0B0DFE881F98130973B
:104DD00021F01083E881F9811182DF91CF911F9139
:104DE00008951F93CF93DF93EC01162F81E090E09D
:104DF0009D838C83CE0161E070E097DFE881F981CB
:104E0000309721F01083E881F9811182DF91CF91F1
:104E10001F9108951F93CF93DF93EC01162F81E02C
:104E200090E09D838C83CE0161E070E07EDFE881BD
:104E3000F981309721F01083E881F9811182DF91A7
:104E4000CF911F9108951F93CF93DF93EC01162FFD
:104E500081E090E09D838C83CE0161E070E065DFAE
:104E6000E881F981309721F01083E881F98111827E
:104E7000DF91CF911F9108950F931F93CF93DF93ED
:104E80008C01EB016C817D81FC01758364834DDFB6
:104E9000F80180819181009721F0688179810E94D9
:104EA0009939DF91CF911F910F9108950F931F931F
:104EB000CF93DF938C01EB016C817D81FC017583C5
:104EC000648333DFF80180819181009721F068814C
:104ED00079810E949939DF91CF911F910F910895A7
:104EE000EF92FF920F931F93DF93CF93CDB7DEB76F
:104EF000A1970FB6F894DEBF0FBECDBF8C01CB01DA
:104F0000BA017E010894E11CF11CA7012AE030E0FF
:104F10000E94503AF70101900020E9F73197EE190D
:104F2000FF09D8011596FC93EE931497C801BF01B1
:104F3000FCDEF80180819181009719F0B7010E9491
:104F40009939A1960FB6F894DEBF0FBECDBFCF91B1
:104F5000DF911F910F91FF90EF900895EF92FF92D4
:104F60000F931F93DF93CF93CDB7DEB7A1970FB603
:104F7000F894DEBF0FBECDBF8C01CB01BA017E011C
:104F80000894E11CF11CA7012AE030E00E94503A8D
:104F9000F70101900020E9F73197EE19FF09D801D8
:104FA0001596FC93EE931497C801BF01BEDEF8017D
:104FB00080819181009719F0B7010E949939A196DB
:104FC0000FB6F894DEBF0FBECDBFCF91DF911F911A
:104FD0000F91FF90EF900895EF92FF920F931F9320
:104FE000DF93CF93CDB7DEB7A1970FB6F894DEBFAE
:104FF0000FBECDBF8C019A0180E090E07E01089445
:10500000E11CF11CA7010E94503AF7010190002019
:10501000E9F73197EE19FF09D8011596FC93EE9345
:105020001497C801BF0181DEF8018081918100974A
:1050300019F0B7010E949939A1960FB6F894DEBF16
:105040000FBECDBFCF91DF911F910F91FF90EF90D9
:105050000895EF92FF920F931F93DF93CF93CDB7F5
:10506000DEB7A1970FB6F894DEBF0FBECDBF8C019F
:105070009A0180E090E07E010894E11CF11CA701F8
:105080000E94503AF70101900020E9F73197EE199C
:10509000FF09D8011596FC93EE931497C801BF0140
:1050A00044DEF80180819181009719F0B7010E94D8
:1050B0009939A1960FB6F894DEBF0FBECDBFCF9140
:1050C000DF911F910F91FF90EF9008950F931F9321
:1050D000CF93DF938C01EB016115710511F4C7EAE1
:1050E000D2E0FE0101900020E9F73197EC1BFD0BA7
:1050F000D8011596FC93EE931497C801BF0115DEF5
:10510000F80180819181009719F0BE010E949939C0
:10511000DF91CF911F910F910895AF92BF92CF92DF
:10512000DF92EF92FF920F931F93CF93DF93B82EEE
:10513000A92E6B01C82FD92FFB0160817181CE018F
:10514000C5DFEE24FF240EC0088119810E0D1F1D3E
:10515000F801808190E00E946239F8018083089410
:10516000E11CF11CF60184819581E816F90660F3D3
:105170008B2D9A2DDF91CF911F910F91FF90EF9082
:10518000DF90CF90BF90AF900895AF92BF92CF9233
:10519000DF92EF92FF920F931F93CF93DF93B82E7E
:1051A000A92E6B01C82FD92FFB0160817181CE011F
:1051B0008DDFEE24FF240EC0088119810E0D1F1D06
:1051C000F801808190E00E945A39F80180830894A8
:1051D000E11CF11CF60184819581E816F90660F363
:1051E0008B2D9A2DDF91CF911F910F91FF90EF9012
:1051F000DF90CF90BF90AF900895EF92FF920F9302
:105200001F93DF93CF93CDB7DEB72C970FB6F894EB
:10521000DEBF0FBECDBFFC017B018617970711F4DF
:1052200001E025C024813581DB0114968D919C918C
:1052300015972817390711F000E019C0CE01019623
:10524000BF01A3DF09811A81CE010796B7019DDF57
:105250006F817885C8010E94903900E0009709F4B9
:1052600001E0CE010796B6DBCE010196B3DB802FBD
:105270002C960FB6F894DEBF0FBECDBFCF91DF9155
:105280001F910F91FF90EF900895CF92DF92EF92D0
:10529000FF921F93CF93DF936C017B01B901241719
:1052A000350710F4BA01A901D70114968D919C918C
:1052B0001597EB018617970708F4EC01D701ED91DC
:1052C000FC911197EC0FFD1F108110826D917C9164
:1052D000640F751FC601FADED701ED91FC91EC0F4A
:1052E000FD1F1083C601DF91CF911F91FF90EF90BA
:1052F000DF90CF9008950F931F938C01FB012481C1
:105300003581C3DFC8011F910F9108958F929F923D
:10531000AF92BF92CF92DF92EF92FF920F931F93C3
:10532000DF93CF9300D000D000D0CDB7DEB75C01C3
:105330006B01DB0114968D919C911597009789F173
:1053400001974817590768F1F5018481958148173D
:10535000590738F5ED91FC9100817A014E010894CE
:10536000811C911C1CC0D501ED91FC91EE0DFF1D1F
:105370008081801789F4F601248135812E0D3F1D2F
:10538000C401B501A70181DFC401B601DDDB182F1F
:10539000C40120DB112341F40894E108F108F7FE71
:1053A000E2CFEE24EA94FE2CC70126960FB6F894BD
:1053B000DEBF0FBECDBFCF91DF911F910F91FF9048
:1053C000EF90DF90CF90BF90AF909F908F90089517
:1053D000FC01DB014481558114968D919C911597B8
:1053E000481B590BCF0192CFAF92BF92CF92DF9261
:1053F000EF92FF920F931F93DF93CF9300D000D0D3
:1054000000D0CDB7DEB75C018B01DB016D917C91E3
:105410006115710519F4B8012FDD3BC0CE0101966D
:1054200055DEF801E480F580CC24DD240EC0D801DF
:10543000ED91FC91EC0DFD1D808190E00E945239B0
:10544000892B31F00894C11CD11CCE14DF0478F3F1
:10545000ED80FE800BC0D801ED91FC91EE0DFF1D9B
:10546000808190E00E945239892B31F00894E10844
:10547000F108CE14DF0478F30894E11CF11CC50197
:105480008E010F5F1F4FB801A6019701FEDEC80114
:10549000A1DAC50126960FB6F894DEBF0FBECDBFC8
:1054A000CF91DF911F910F91FF90EF90DF90CF9000
:1054B000BF90AF9008952F923F924F925F926F925C
:1054C0007F928F929F92AF92BF92CF92DF92EF9294
:1054D000FF920F931F93DF93CF93CDB7DEB76897FB
:1054E0000FB6F894DEBF0FBECDBF3C01FB012A0111
:1054F0001901608171816115710519F4BF01BCDC6E
:105500004CC07E010894E11CF11CC701DFDD8E0157
:10551000095F1F4FC80167EA72E0D8DDD02EC12EA7
:105520003DE0832E912C8C0E9D1E23E1A22EB12CEA
:10553000AC0EBD1E1DC0C401B70140E050E0980193
:10554000A4DE8D2D9C2DB401B7DBC40143DA8D2D73
:105550009C2DB101B1DBF20144815581400F511FF7
:10556000C501B701C8DEC701B501F3DBC50132DAF9
:10557000C701B201C7DA8C01FFEF8F3F9F07D9F651
:105580008D2D9C2DB70198DBC3016D2D7C2D74DC16
:105590008D2D9C2D1FDAC7011DDAC30168960FB649
:1055A000F894DEBF0FBECDBFCF91DF911F910F9159
:1055B000FF90EF90DF90CF90BF90AF909F908F9033
:1055C0007F906F905F904F903F902F900895EF9253
:1055D000FF920F931F93DF93CF9300D000D000D0A2
:1055E000CDB7DEB77C01FB01142F022F60817181E2
:1055F0006115710519F4BF013FDC16C0CE0101969B
:1056000065DD89819A8101C00083612F70E00E946D
:105610008539FC010097C1F7C7018E010F5F1F4F4D
:10562000B8012ADCC801D6D9C70126960FB6F8946E
:10563000DEBF0FBECDBFCF91DF911F910F91FF90C5
:10564000EF9008950F931F93CF93DF938C01EB019D
:105650006115710511F4C7EAD2E0FE010190002046
:10566000E9F73197EC1BFD0BD8011596FC93EE93EF
:105670001497C801BF0159DBF8018081918100971F
:1056800019F0BE010E949939DF91CF911F910F91BE
:105690000895EF92FF920F931F93DF93CF93CDB7AF
:1056A000DEB7A1970FB6F894DEBF0FBECDBF8C0159
:1056B000CB01BA017E010894E11CF11CA7010E94F4
:1056C000013AF70101900020E9F73197EE19FF093F
:1056D000D8011596FC93EE931497C801BF0125DB02
:1056E000F80180819181009719F0B7010E949939E2
:1056F000A1960FB6F894DEBF0FBECDBFCF91DF915C
:105700001F910F91FF90EF900895EF92FF920F93EA
:105710001F93DF93CF93CDB7DEB7A1970FB6F89461
:10572000DEBF0FBECDBF8C01CB01BA017E01089454
:10573000E11CF11CA7010E94013AF7010190002031
:10574000E9F73197EE19FF09D8011596FC93EE930E
:105750001497C801BF01E9DAF801808191810097AF
:1057600019F0B7010E949939A1960FB6F894DEBFDF
:105770000FBECDBFCF91DF911F910F91FF90EF90A2
:105780000895EF92FF920F931F93DF93CF93CDB7BE
:10579000DEB7A1970FB6F894DEBF0FBECDBF8C0168
:1057A000CB017E010894E11CF11CB7010E94E23993
:1057B000F70101900020E9F73197EE19FF09D801B0
:1057C0001596FC93EE931497C801BF01AEDAF80169
:1057D00080819181009719F0B7010E949939A196B3
:1057E0000FB6F894DEBF0FBECDBFCF91DF911F91F2
:1057F0000F91FF90EF900895EF92FF920F931F93F8
:10580000DF93CF93CDB7DEB7A1970FB6F894DEBF85
:105810000FBECDBF8C01CB017E010894E11CF11CB1
:10582000B7010E94E239F70101900020E9F73197B2
:10583000EE19FF09D8011596FC93EE931497C80151
:10584000BF0173DAF80180819181009719F0B701E7
:105850000E949939A1960FB6F894DEBF0FBECDBF56
:10586000CF91DF911F910F91FF90EF9008951F92BC
:105870000F920FB60F9211242F933F938F939F9304
:10588000AF93BF938091A4059091A505A091A60523
:10589000B091A7053091A8050196A11DB11D232F38
:1058A0002D5F2D3720F02D570196A11DB11D20939E
:1058B000A8058093A4059093A505A093A605B09391
:1058C000A7058091A0059091A105A091A205B09196
:1058D000A3050196A11DB11D8093A0059093A1057C
:1058E000A093A205B093A305BF91AF919F918F9113
:1058F0003F912F910F900FBE0F901F9018958FB76B
:10590000F8942091A4053091A5054091A6055091E9
:10591000A7058FBFB901CA0108959FB7F8942091D8
:10592000A0053091A1054091A2055091A30586B52F
:10593000A89B06C08F3F21F02F5F3F4F4F4F5F4F17
:105940009FBF542F432F322F2227280F311D411D77
:10595000511D82E0220F331F441F551F8A95D1F736
:10596000B901CA010895EF92FF920F931F93CF934D
:10597000DF937B018C01D1DFEB010DC0CEDF6C1B0F
:105980007D0B685E7340D0F30894E108F1080109CB
:105990001109C851DC4FE114F1040105110571F73B
:1059A000DF91CF911F910F91FF90EF900895019794
:1059B00039F0880F991F880F991F02970197F1F707
:1059C0000895789484B5826084BD84B5816084BD77
:1059D00085B5826085BD85B5816085BDEEE6F0E068
:1059E000808181608083E1E8F0E0108280818260C4
:1059F0008083808181608083E0E8F0E08081816045
:105A00008083E1EBF0E0808184608083E0EBF0E074
:105A1000808181608083EAE7F0E080818460808318
:105A200080818260808380818160808380818068C2
:105A300080831092C10008958093A8020895982F42
:105A40008E3008F09E5097708091A8028295880F42
:105A5000880F807C892B80937C0080917A00806401
:105A600080937A0080917A0086FDFCCF20917800A7
:105A700040917900942F80E030E0282B392BC90128
:105A800008951F93CF93DF93182FEB0161E057D058
:105A9000209709F44AC0CF3FD10509F449C0E12F4E
:105AA000F0E0E357FD4F84918330C1F0843028F457
:105AB000813051F08230B1F50CC0863019F1873059
:105AC00049F1843079F514C084B5806884BDC7BDC0
:105AD00032C084B5806284BDC8BD2DC08091800075
:105AE000806880938000D0938900C093880023C091
:105AF00080918000806280938000D0938B00C0935F
:105B00008A0019C08091B00080688093B000C09373
:105B1000B30011C08091B00080628093B000C09348
:105B2000B40009C0C038D1051CF4812F60E002C068
:105B3000812F61E057D0DF91CF911F910895482FB9
:105B400050E0CA0187589D4FFC0124914B595D4F8D
:105B5000FA0184918823C1F0E82FF0E0EE0FFF1FD7
:105B6000E95BFD4FA591B491662341F49FB7F8948A
:105B70008C91209582238C939FBF08959FB7F894B2
:105B80008C91822B8C939FBF0895833071F0843069
:105B900028F48130A1F0823021F514C08630B1F0B4
:105BA0008730D1F08430E9F404C0809180008F7791
:105BB00003C0809180008F7D80938000089584B51C
:105BC0008F7702C084B58F7D84BD08958091B00029
:105BD0008F778093B00008958091B0008F7D80937F
:105BE000B0000895FF920F931F93F62E482F50E0B8
:105BF000CA0183579D4FFC012491CA0187589D4FCC
:105C0000FC0114914B595D4FFA0104910023D1F02E
:105C1000222311F0822FB9DFE02FF0E0EE0FFF1FFB
:105C2000EF5AFD4FA591B491FF2031F49FB7F8943E
:105C30008C911095812304C09FB7F8948C91812B8F
:105C40008C939FBF1F910F91FF9008950F931F9307
:105C5000482F50E0CA0183579D4FFC012491CA018F
:105C600087589D4FFC0104914B595D4FFA011491E7
:105C7000112319F420E030E014C0222311F0822F08
:105C800084DF812F90E0880F991F855A9D4FFC017A
:105C9000A591B4918C9120E030E0802311F021E0B7
:105CA00030E0C9011F910F910895EF92FF920F9379
:105CB0001F937B018C0120E030E040E05FE4ABD338
:105CC00088237CF0C801B70120E030E040E05FE4C9
:105CD0005ED151D49B01AC0120503040404050482F
:105CE00005C0C801B70147D49B01AC01B901CA0185
:105CF0001F910F91FF90EF900895A0E0B0E0E2E8CF
:105D0000FEE284C7DC012B01FA019C91923008F479
:105D100039C1EB018881823008F433C1943069F4D1
:105D2000843009F02FC111969C91119789819817A1
:105D300009F428C1A9EAB2E025C1843009F421C1DF
:105D40008230A9F4923009F01DC19A01AD0188E0BA
:105D5000EA010990AE01E90109929E018150C1F763
:105D6000E201898111969C918923818308C1923037
:105D700009F407C112962D903C901397EB018A818C
:105D80009B811496AD90BD90CD90DC901797EC80E0
:105D9000FD800E811F819101281B390BB90137FF4E
:105DA00004C066277727621B730B603271050CF005
:105DB00061C0121613066CF537014801062E04C0A7
:105DC00096948794779467940A94D2F721E030E010
:105DD00040E050E004C0220F331F441F551F6A9556
:105DE000D2F721503040404050402E213F214023E7
:105DF0005123211531054105510521F021E030E005
:105E000040E050E079018A01E628F728082919299D
:105E10003CC0232BD1F1260E371E35014601062E3C
:105E200004C096948794779467940A94D2F721E0FB
:105E300030E040E050E004C0220F331F441F551FE4
:105E40006A95D2F721503040404050402A213B21F2
:105E50004C215D21211531054105510521F021E03D
:105E600030E040E050E059016A01A628B728C82870
:105E7000D9280BC0821593052CF01C01AA24BB2441
:105E8000650103C0EE24FF24870111969C91D20185
:105E900011968C91981709F445C0992339F0A801FF
:105EA00097012A193B094C095D0906C0A601950115
:105EB0002E193F09400B510B57FD08C01182338248
:105EC000228224833583468357831DC081E08183EA
:105ED0003382228288279927DC01821B930BA40B33
:105EE000B50B84839583A683B7830DC0220F331F20
:105EF000441F551F248335834683578382819381B2
:105F00000197938382832481358146815781DA0109
:105F1000C9010197A109B1098F5F9F4FAF4FBF43DF
:105F200028F30BC0918333822282EA0CFB1C0C1DE8
:105F30001D1DE482F5820683178383E0808324811C
:105F400035814681578157FF1AC0C901AA2797FD9D
:105F5000A095BA2F81709070A070B070569547953B
:105F600037952795822B932BA42BB52B8483958370
:105F7000A683B78382819381019693838283DF0115
:105F800001C0D201CD01CDB7DEB7E2E15BC6A0E230
:105F9000B0E0ECECFFE246C669837A838B839C8396
:105FA0002D833E834F835887E9E0EE2EF12CEC0ED3
:105FB000FD1ECE010196B701C9D48E010F5E1F4FA1
:105FC000CE010596B801C2D48A8991E089278A8BCF
:105FD000C701B801AE01475E5F4F8FDEE1D3A096E7
:105FE000E6E03CC6A0E2B0E0E7EFFFE21BC6698353
:105FF0007A838B839C832D833E834F835887F9E07C
:10600000EF2EF12CEC0EFD1ECE010196B7019ED4B1
:106010008E010F5E1F4FCE010596B80197D4C701C0
:10602000B801AE01475E5F4F68DEBAD3A096E6E0E6
:1060300015C6A0E2B0E0EEE1F0E3E8C569837A833B
:106040008B839C832D833E834F835887CE0101969B
:10605000BE01675F7F4F7AD4CE010596BE016F5EA9
:106060007F4F74D49985923088F089898230C8F046
:10607000943019F4823051F404C0843029F4923001
:1060800081F489EA92E0C6C0923049F420E09A8512
:106090008A89981321E02A87CE010996BBC08230F5
:1060A00049F420E09A858A89981321E02A8BCE0151
:1060B0004196B0C02D843E844F8458886D887E8878
:1060C0008F88988CEE24FF248701AA24BB246501C5
:1060D00040E050E060E070E0E0E0F0E0C10181709D
:1060E0009070892BE9F0E60CF71C081D191D9A0128
:1060F000AB012A0D3B1D4C1D5D1D80E090E0A0E032
:10610000B0E0E614F7040805190520F481E090E0FA
:10611000A0E0B0E0BA01A901480F591F6A1F7B1F18
:10612000AA0CBB1CCC1CDD1C97FE08C081E090E0D3
:10613000A0E0B0E0A82AB92ACA2ADB2A3196E032C8
:10614000F10549F0660C771C881C991C56944794FD
:1061500037942794C3CFFA85EA892B893C898B85AC
:106160009C85280F391F2E5F3F4F17C0CA018170D1
:106170009070892B61F016950795F794E79480E06D
:1061800090E0A0E0B0E8E82AF92A0A2B1B2B7695CC
:106190006795579547952F5F3F4F77FDE7CF0CC029
:1061A000440F551F661F771F17FD4160EE0CFF1C43
:1061B000001F111F21503040403090E0590790E0FF
:1061C000690790E4790760F32B8F3C8FDB01CA01EC
:1061D0008F779070A070B07080349105A105B105E3
:1061E00061F447FD0AC0E114F1040105110529F02D
:1061F000405C5F4F6F4F7F4F40781A8EFE1711F053
:1062000081E08A8F4D8F5E8F6F8F78A383E0898FB7
:10621000CE014996C5D2A096E2E114C5A8E1B0E04E
:10622000E3E1F1E3FBC469837A838B839C832D8351
:106230003E834F835887B9E0EB2EF12CEC0EFD1E08
:10624000CE010196B70182D38E010F5E1F4FCE01A2
:106250000596B8017BD32985223008F47EC03989A0
:10626000323010F4B8017CC08A859A8989278A87E0
:10627000243011F0223031F4231709F06EC069EA9E
:1062800072E06EC0343039F41D861E861F86188A6F
:106290001C861B8604C0323021F484E08987B70154
:1062A0005FC02B853C858B899C89281B390B3C87DB
:1062B0002B87ED84FE840F851889AD88BE88CF8832
:1062C000D88CEA14FB040C051D0540F4EE0CFF1CF1
:1062D000001F111F215030403C872B8720E030E009
:1062E00040E050E080E090E0A0E0B0E460E070E0EA
:1062F000EA14FB040C051D0540F0282B392B4A2B12
:106300005B2BEA18FB080C091D09B695A795979514
:106310008795EE0CFF1C001F111F6F5F7F4F6F31C1
:10632000710531F7DA01C9018F779070A070B070F4
:1063300080349105A105B10561F427FD0AC0E1147F
:10634000F1040105110529F0205C3F4F4F4F5F4FCD
:1063500020782D873E874F87588BBE01675F7F4F20
:10636000CB011ED26896EAE075C4A8E1B0E0EAEB82
:10637000F1E358C469837A838B839C832D833E83A6
:106380004F83588789E0E82EF12CEC0EFD1ECE01DC
:106390000196B701DBD28E010F5E1F4FCE0105962D
:1063A000B801D4D28985823038F08989823020F0D2
:1063B000C701B80143D301C081E06896E6E04EC44E
:1063C000A8E1B0E0E5EEF1E32DC469837A838B8325
:1063D0009C832D833E834F83588789E0E82EF12CE0
:1063E000EC0EFD1ECE010196B701B0D28E010F5EFC
:1063F0001F4FCE010596B801A9D28985823038F0A9
:106400008989823020F0C701B80118D301C08FEF0D
:106410006896E6E023C4A8E1B0E0E0E1F2E302C45C
:1064200069837A838B839C832D833E834F83588734
:1064300089E0E82EF12CEC0EFD1ECE010196B7018D
:1064400085D28E010F5E1F4FCE010596B8017ED218
:106450008985823038F08989823020F0C701B801FF
:10646000EDD201C08FEF6896E6E0F8C3A8E1B0E096
:10647000EBE3F2E3D7C369837A838B839C832D8319
:106480003E834F83588789E0E82EF12CEC0EFD1EE9
:10649000CE010196B7015AD28E010F5E1F4FCE0179
:1064A0000596B80153D28985823038F089898230C7
:1064B00020F0C701B801C2D201C081E06896E6E0D1
:1064C000CDC3A8E0B0E0E6E6F2E3A9C39B01AC01CE
:1064D00083E08983DA01C9018827B7FD839599276D
:1064E000AA27BB27B82E211531054105510519F4FE
:1064F00082E0898339C08823A9F0203080E0380702
:1065000080E0480780E8580729F460E070E080E008
:106510009FEC2EC0EE24FF248701E21AF30A040B3D
:10652000150B02C079018A018EE1C82ED12CDC82C4
:10653000CB82ED82FE820F831887C801B701E1D0BC
:1065400001971816190684F4082E04C0EE0CFF1CDF
:10655000001F111F0A94D2F7ED82FE820F83188765
:10656000C81AD90ADC82CB82BA82CE01019618D130
:106570002896E9E070C3ACE0B0E0E0ECF2E356C38B
:1065800069837A838B839C83CE010196BE016B5F06
:106590007F4FDCD18D81823061F1823050F18430C7
:1065A00021F48E81882351F12EC02F81388537FD4B
:1065B00020C06E812F3131051CF06623F9F023C015
:1065C0008EE190E0821B930B29853A854B855C8593
:1065D00004C056954795379527958A95D2F7662337
:1065E000B1F050954095309521953F4F4F4F5F4FFB
:1065F0000EC020E030E040E050E009C02FEF3FEF58
:106600004FEF5FE704C020E030E040E050E8B90120
:10661000CA012C96E2E026C3A8E0B0E0E1E1F3E392
:10662000FDC27B018C01611571058105910519F48D
:1066300082E089835FC083E089838EE1C82ED12CFC
:10664000DC82CB82ED82FE820F831887C801B701FE
:1066500058D0FC013197F7FF3BC0222733272E1B70
:106660003F0B57016801022E04C0D694C794B7941B
:10667000A7940A94D2F740E050E060E070E081E037
:1066800090E0A0E0B0E004C0880F991FAA1FBB1FD4
:106690002A95D2F70197A109B1098E219F21A02344
:1066A000B1230097A105B10521F041E050E060E081
:1066B00070E04A295B296C297D294D835E836F83B5
:1066C00078878EE190E08E1B9F0B9C838B8312C09A
:1066D000309781F00E2E04C0EE0CFF1C001F111F1E
:1066E0000A94D2F7ED82FE820F831887CE1ADF0A52
:1066F000DC82CB821A82CE01019652D02896EAE043
:10670000A9C2EF92FF920F931F937B018C0180E04F
:10671000E81680E0F80681E0080780E0180788F4B2
:106720008FEFE816F1040105110531F028F088E03B
:1067300090E0A0E0B0E017C080E090E0A0E0B0E022
:1067400012C080E0E81680E0F80680E0080781E0EB
:10675000180728F088E190E0A0E0B0E004C080E1F4
:1067600090E0A0E0B0E020E230E040E050E0281B04
:10677000390B4A0B5B0B04C016950795F794E79409
:106780008A95D2F7F701EF54FD4F8081281B31091C
:1067900041095109C9011F910F91FF90EF90089590
:1067A000DF92EF92FF920F931F93FC01E480F5803C
:1067B00006811781D1808081823058F480E090E09A
:1067C000A0E1B0E0E82AF92A0A2B1B2BEFEFF0E05A
:1067D000A6C0843009F49EC0823019F4E0E0F0E0F5
:1067E0009BC0E114F1040105110519F4E0E0F0E0AB
:1067F00096C0628173819FEF623879070CF05BC0AD
:1068000022E83FEF261B370B2A3131052CF020E020
:1068100030E040E050E02AC0B801A701022E04C0D9
:1068200076956795579547950A94D2F781E090E061
:10683000A0E0B0E004C0880F991FAA1FBB1F2A95D3
:10684000D2F70197A109B1098E219F21A023B1237D
:106850000097A105B10521F081E090E0A0E0B0E053
:106860009A01AB01282B392B4A2B5B2BDA01C9018A
:106870008F779070A070B07080349105A105B1053C
:1068800039F427FF09C0205C3F4F4F4F5F4F04C0D2
:10689000215C3F4F4F4F5F4FE0E0F0E02030A0E041
:1068A0003A07A0E04A07A0E45A0710F0E1E0F0E060
:1068B00079018A0127C06038710564F5FB01E15850
:1068C000FF4FD801C7018F779070A070B0708034EF
:1068D0009105A105B10539F4E7FE0DC080E490E013
:1068E000A0E0B0E004C08FE390E0A0E0B0E0E80EEC
:1068F000F91E0A1F1B1F17FF05C016950795F79471
:10690000E794319687E016950795F794E7948A9572
:10691000D1F705C0EFEFF0E0EE24FF2487016E2FE2
:10692000679566276795902F9F77D794DD24D79436
:106930008E2F8695492F462B582F5D29B701CA0106
:106940001F910F91FF90EF90DF900895FC01DB0104
:10695000408151812281622F6F7770E0221F2227B0
:10696000221F9381892F880F822B282F30E0991FB7
:106970009927991F11969C93119721153105A9F517
:10698000411551056105710511F482E037C082E8B7
:106990009FEF13969C938E9312979A01AB0167E039
:1069A000220F331F441F551F6A95D1F783E08C9344
:1069B0000DC0220F331F441F551F12968D919C91BD
:1069C0001397019713969C938E931297203080E033
:1069D000380780E0480780E4580758F314962D9351
:1069E0003D934D935C93179708952F3F310579F4AC
:1069F000411551056105710519F484E08C930895E2
:106A000064FF03C081E08C9312C01C9210C02F570A
:106A1000304013963C932E93129783E08C9387E03B
:106A2000440F551F661F771F8A95D1F7706414961F
:106A30004D935D936D937C93179708951F93DC019D
:106A4000FB019C91923008F447C08081823008F4A9
:106A500043C0943051F411961C91843099F5818192
:106A6000682F70E0611B71093FC0843021F09230C3
:106A700031F48230B9F18181882389F12DC01196DA
:106A80001C9111978230F1F081811817D9F4129678
:106A90002D913C911397828193818217930794F0F3
:106AA00028173907BCF014968D919D910D90BC91DB
:106AB000A02D2481358146815781281739074A073F
:106AC0005B0718F4112341F00AC082179307A4074B
:106AD000B50740F4112319F061E070E005C06FEFD5
:106AE0007FEF02C060E070E0CB011F910895629FCC
:106AF000D001739FF001829FE00DF11D649FE00DB6
:106B0000F11D929FF00D839FF00D749FF00D659F16
:106B1000F00D9927729FB00DE11DF91F639FB00D15
:106B2000E11DF91FBD01CF0111240895991B79E0E2
:106B300004C0991F961708F0961B881F7A95C9F70D
:106B40008095089597FB092E07260AD077FD04D07B
:106B500049D006D000201AF4709561957F4F0895B2
:106B6000F6F7909581959F4F0895A1E21A2EAA1BE2
:106B7000BB1BFD010DC0AA1FBB1FEE1FFF1FA217ED
:106B8000B307E407F50720F0A21BB30BE40BF50BEA
:106B9000661F771F881F991F1A9469F76095709573
:106BA000809590959B01AC01BD01CF01089597FBA5
:106BB000092E05260ED057FD04D0D7DF0AD0001CC1
:106BC00038F450954095309521953F4F4F4F5F4F8A
:106BD0000895F6F790958095709561957F4F8F4F4A
:106BE0009F4F0895AA1BBB1B51E107C0AA1FBB1FE3
:106BF000A617B70710F0A61BB70B881F991F5A9549
:106C0000A9F780959095BC01CD0108952F923F92F0
:106C10004F925F926F927F928F929F92AF92BF92AC
:106C2000CF92DF92EF92FF920F931F93CF93DF9358
:106C3000CDB7DEB7CA1BDB0B0FB6F894DEBF0FBEB5
:106C4000CDBF09942A88398848885F846E847D8402
:106C50008C849B84AA84B984C884DF80EE80FD8004
:106C60000C811B81AA81B981CE0FD11D0FB6F8947A
:106C7000DEBF0FBECDBFED010895EE0FFF1F0590E3
:106C8000F491E02D09944ED080F09F3740F491119B
:106C90000EF460C060E070E080E89FE3089526F0A5
:106CA0001B16611D711D811D14C02EC03BD080F0CC
:106CB0009F3740F491110EF04DC060E070E080E825
:106CC0009FEB089526F41B16611D711D811D01C0E7
:106CD0001BC0882371F4772321F09850872B762FDF
:106CE00007C0662311F499270DC09051862B70E0E0
:106CF00060E02AF09A95660F771F881FDAF7880FF1
:106D00009695879597F908959F3F31F0915020F41B
:106D1000879577956795B795880F911D9695879577
:106D200097F9089525D0A0F0BEE7B91788F4BB27DE
:106D30009F3860F41616B11D672F782F8827985F4B
:106D4000F7CF869577956795B11D93959639C8F3DA
:106D50000895E894BB2766277727CB0197F9089514
:106D600057FD9058440F551F59F05F3F71F04795FC
:106D7000880F97FB991F61F09F3F79F087950895E1
:106D8000121613061406551FF2CF4695F1DF08C000
:106D9000161617061806991FF1CF8695710561051D
:106DA000089408950F931F93CF93DF93689F8001FA
:106DB000699F100D789F100D1124C8010DD0EC01B2
:106DC000009721F060E070E0A8018DD2CE01DF9144
:106DD000CF911F910F910895CF93DF93BC01823023
:106DE000910510F462E070E0A091AB05B091AC05A4
:106DF000ED01E0E0F0E040E050E021C088819981C1
:106E00008617970769F48A819B81309719F09383DD
:106E1000828304C09093AC058093AB05FE0134C01F
:106E20006817790738F44115510519F0841795074B
:106E300008F4AC01FE018A819B819C01E901209745
:106E4000E9F641155105A9F1CA01861B970B049774
:106E500008F4BA01E0E0F0E02AC08D919C9111970E
:106E600084179507F9F46417750781F412968D91CC
:106E70009C911397309719F09383828304C0909369
:106E8000AC058093AB05FD0132964FC0CA01861B4D
:106E9000970BFD01E80FF91F6193719302978D9392
:106EA0009C9343C0FD01828193819C01D90110977D
:106EB000A1F68091A9059091AA05892B41F48091B2
:106EC000B3039091B4039093AA058093A9054091D0
:106ED000B5035091B6034115510541F44DB75EB766
:106EE0008091B1039091B203481B590B2091A905E1
:106EF0003091AA0524173507B0F4CA01821B930B01
:106F00008617970780F0AB014E5F5F4F8417950798
:106F100050F0420F531F5093AA054093A905F90161
:106F20006193719302C0E0E0F0E0CF01DF91CF9177
:106F30000895CF93DF93009709F450C0EC01229796
:106F40001B821A82A091AB05B091AC05109709F194
:106F500040E050E0AC17BD0708F1BB83AA83FE01F7
:106F600021913191E20FF31FAE17BF0779F48D9194
:106F70009C911197280F391F2E5F3F4F398328832B
:106F800012968D919C9113979B838A83411551058D
:106F900071F4D093AC05C093AB0520C012968D91CF
:106FA0009C911397AD01009711F0DC01D3CFFA014A
:106FB000D383C28321913191E20FF31FCE17DF07F4
:106FC00069F488819981280F391F2E5F3F4FFA019C
:106FD000318320838A819B8193838283DF91CF9148
:106FE0000895A0E0B0E0E6EFF7E318CEEC01A8804A
:106FF000B980CA80DB80A114B104C104D10441F47A
:1070000084E2A82E89EDB82E8BE5C82E87E0D82E15
:10701000C601B5012DE133EF41E050E0C8DD27EABC
:1070200031E440E050E063DD7B018C01C601B50135
:107030002DE133EF41E050E0BADDCA01B9012CEE99
:1070400034EF4FEF5FEF53DD6E0D7F1D801F911FFB
:1070500097FF04C0615070408040904868837983F6
:107060008A839B839B01AC015F77B901CA01CDB7CD
:10707000DEB7EAE0EFCDB5CF87EB93E0B2CF609318
:10708000B7037093B8038093B9039093BA0308953C
:10709000A0E0B0E0EDE4F8E3BFCD8C01009721F46F
:1070A000CB019ADE8C01B6C09EEFE92E9FEFF92E40
:1070B000E00EF11E5801A60EB71EAE14BF0408F470
:1070C000A7C08EEF882E8FEF982E8A0C9B1CE701AD
:1070D0004881598146175707B0F04530510508F4EB
:1070E00099C0CA0104978617970708F493C04250C5
:1070F0005040461B570BF4015183408379836883CA
:10710000C50117DF87C06B01C41AD50AE091AB0532
:10711000F091AC05A0E0B0E0C0E0D0E042C0E815DE
:10712000F905A1F5208131812C153D0578F1C901C2
:1071300002968C159D05A8F04E5F5F4F420F531FBE
:10714000E7015983488322813381109729F01396F0
:107150003C932E9312975EC03093AC052093AB0501
:1071600059C0225030402C193D093183208310979B
:1071700029F01396FC93EE93129704C0F093AC059C
:10718000E093AB05F7017183608344C080819181F6
:10719000C817D90708F4EC01DF01828193819C01B3
:1071A000F901309709F0BBCF400F511F8091A9051D
:1071B0009091AA0584179507E9F4C617D707D0F46C
:1071C0002091B5033091B6032115310541F42DB757
:1071D0003EB78091B1039091B203281B390BA216E0
:1071E000B306B0F4B092AA05A092A905E70179838D
:1071F000688310C0CB01F0DDEC01009749F0F70186
:1072000040815181B80166D0C80193DE8E0102C071
:1072100000E010E0C801CDB7DEB7ECE019CDFC010D
:1072200088279927E89421912032E9F3293010F03A
:107230002E30C8F32B3239F02D3231F4689403C06C
:1072400027D1820F911D219120532A30C8F31EF4BB
:10725000909581959F4F08951F93FC01992788274A
:10726000BC01E89411911032E9F3193010F01E308E
:10727000C8F31B3249F01D3241F4689405C0F3D0C5
:10728000610F711D811D911D119110531A30B8F3BA
:107290003EF490958095709561957F4F8F4F9F4FED
:1072A0001F910895911135C1803219F08950855090
:1072B000D0F708959111089581548A5108F4805EA1
:1072C000855A08959111089581568A5108F4805283
:1072D00085580895FB01DC0102C001900D924150D8
:1072E0005040D8F70895DC0101C06D9341505040E3
:1072F000E0F70895FB01DC010D900020E9F71197FC
:1073000001900D920020E1F70895FC01819186170C
:1073100021F08823D9F7992708953197CF0108954F
:10732000FB01DC018D91019080190110D9F3990BBB
:107330000895FB01DC0101900D920020E1F7089512
:10734000FB01DC014150504030F08D9101908019DB
:1073500019F40020B9F7881B990B0895FB01DC0193
:107360004150504048F001900D920020C9F701C0F3
:107370001D9241505040E0F70895FC0181E090E0FB
:107380000190061609F4CF010020D1F70197089566
:10739000FB0151915523A9F0BF01DC014D91451727
:1073A0004111E1F759F4CD010190002049F04D91D0
:1073B00040154111C9F3FB014111EFCF81E090E08D
:1073C00001970895FB019F01E8944230BCF04532DB
:1073D000ACF44A3029F497FB1EF4909581959F4FA9
:1073E000642F7727FFDB805D8A330CF0895D819302
:1073F000CB010097A9F716F45DE251931082C90101
:107400008BC0FA01CF93FF93EF9322303CF12532EA
:107410002CF5C22FE894CA3049F497FB3EF49095BE
:107420008095709561957F4F8F4F9F4F2C2F3327FD
:1074300044275527FF93EF9398DBEF91FF91605D11
:107440006A330CF0695D6193B901CA016050704004
:107450008040904059F716F4CDE2C19310828F918D
:107460009F91CF9159C0592F482F372F262F660F44
:10747000771F881F991F660F771F881F991F620F3C
:10748000731F841F951F660F771F881F991F08950C
:107490007AE0979F902D879F802D910D112408955C
:1074A000FA01CF93FF93EF932230C4F02532B4F466
:1074B000C22F2C2F332744275527FF93EF9355DBFB
:1074C000EF91FF91605D6A330CF0695D6193B901E2
:1074D000CA01605070408040904059F710828F91EF
:1074E0009F91CF9119C0F999FECF92BD81BDF89AB5
:1074F000992780B50895262FF999FECF1FBA92BD1E
:1075000081BD20BD0FB6F894FA9AF99A0FBE019684
:107510000895992788270895DC01FC01672F719150
:107520007723E1F7329704C07C916D937083629169
:0C753000AE17BF07C8F30895F894FFCF12
:10753C00200043616C426F6F73743A20000200505C
:10754C0049442000203020302030204D0003003BE7
:10755C00003A004D756C7469446973706C617920E4
:10756C00312E312100000001000A000B006400657F
:10757C00006E006F0004000B0002000600070008FC
:10758C00000900020020002E0080C094D4FF01FFEF
:10759C000001FFFE000103FF000103FF00FF0202D8
:1075AC0000FF030100FF0301000101FF00FF03FFC7
:1075BC0000FF03FF00FF02FF0002FF0200FF0202B8
:1075CC00000202FF00FEFFFE000202FF00FF02FFAE
:1075DC0000FEFFFE00FF02FF00FEFEFF00010203A3
:1075EC00000203FE00010203000102030002FEFE82
:1075FC000002020200010203000202020001020367
:10760C000001020300FFFEFF00FEFFFE000102FF6F
:10761C0000FE02FF00FF020200FF020200FF020355
:10762C0000FE02FF00FF02FF00FFFEFF00FFFEFF57
:10763C0000FEFFFE00FFFEFE00FEFEFF00FEFFFE52
:10764C0000FEFEFF00FFFEFF00FEFFFE00FFFEFF40
:10765C00000406FF000406050006060600040606E4
:10766C000004060500FE06FE0006060500040605DD
:10767C0000FE06FE0004060500FEFE0600000000EB
:10768C0000E011E01100000000061D881C821C3B6C
:10769C001D3A00000000006D1D8A1D2D0020000009
:1076AC00000000FE1E7A1E00000000BB20082120F6
:1076BC002160208B207120AF2000000000E0110819
:1076CC00212021E011E011E011E0112E000000005A
:1076DC0000E0110821202100010000000000000042
:1076EC000000010202030303030404040404040461
:1076FC00040505050505050505050505050505052F
:10770C00050606060606060606060606060606060E
:10771C0006060606060606060606060606060606FD
:10772C0006070707070707070707070707070707DE
:10773C0007070707070707070707070707070707CD
:10774C0007070707070707070707070707070707BD
:10775C0007070707070707070707070707070707AD
:10776C00070808080808080808080808080808088E
:10777C00080808080808080808080808080808087D
:10778C00080808080808080808080808080808086D
:10779C00080808080808080808080808080808085D
:1077AC00080808080808080808080808080808084D
:1077BC00080808080808080808080808080808083D
:1077CC00080808080808080808080808080808082D
:1077DC00080808080808080808080808080808081D
:0C77EC00082000AD0500000100000000B6
:00000001FF
